:100000000C94690D0C94910D0C94910D0C94910D20
:100010000C94910D0C94910D0C94910D0C94910DE8
:100020000C94910D0C94910D0C94C32A0C94352BC7
:100030000C94910D0C94910D0C94910D0C94910DC8
:100040000C94910D0C9415170C94910D0C94910D2A
:100050000C94910D0C94910D0C94910D0C94CB1665
:100060000C94910D0C94910D0C94910D0C94910D98
:100070000C94910D0C94910D0C94910D0C94910D88
:100080000C9440180C94910D0C94910D0C94910DBE
:100090000C94910D0C94910D0C94910D0C94910D68
:1000A0000C94910D0C94910D0C94910D0608002662
:1000B00040402600FFFFFFFFFFFF060800067070AC
:1000C0000600FFFFFFFFFFFF060800000000000022
:1000D0000F9AF1F11A0F03080000006E7A0E07085C
:1000E000000C1C381C0C000C1E3E7C3E1E0C07082D
:1000F000001800000000003C7E7EC3C3663C080878
:10010000000008000000000000387C7E7D390000FF
:100110000808007C7E0E060606007CFEFF7F0F0F9F
:100120000F0606100000FEFE0000000003030000A2
:1001300000FEFFFFFE0004477F7F47049009001484
:1001400091270028904500148180F0180E140007B4
:100150000E1300130805000C010709030011090D17
:1001600007FF180E1400070E130013080500020EF7
:100170000C0212FF180E1400070E130013080500DE
:10018000020E0E0C0511010D07FF90430096800032
:10019000329043914A01C88081F0901800C880F0E5
:1001A000101000F82442F181E1F1E1013519020457
:1001B000F8000000013E60D9999D86869A9CE01067
:1001C0000F0000F8FCFEFFFFFFFFFFFFFFFFFEFC3C
:1001D000F8000000013F7FFFFFFFFFFFFFFFFF1F51
:1001E0000F0000F04884E202C2E2C2026A32040850
:1001F000F00000011AE499839B9B9D9C9C8098D8F9
:10020000271800F0F8FCFEFEFEFEFEFEFEFEFCF8E7
:10021000F00000011BFFFFFFFFFFFFFFFFFFFFFFDD
:100220003F1800E01864020202020202020264188F
:10023000E0000007788890B0B0B0B0B09090C032C5
:100240000D0000E0F8FCFEFEFEFEFEFEFEFEFCF8E9
:10025000E00000077FFFFFFFFFFFFFFFFFFFFF3F03
:100260000D00F008046281810181810181816204B5
:10027000F8000F106C86919B9ABBBBA29B99EE1065
:100280000F00F0F8FCFEFFFFFFFFFFFFFFFFFEFC8B
:10029000F8000F1F7FFFFFFFFFFFFFFFFFFFFF1FA4
:1002A0000F00F04884E202C2E2C2026A320408F09F
:1002B0000000252644419B839B9D9C9C9880985BD5
:1002C0002418F0F8FCFEFEFEFEFEFEFEFEFCF8F03A
:1002D00000003D3F7F7FFFFFFFFFFFFFFFFFFF7F2E
:1002E0003C1800F00C320101010101010101320C46
:1002F000F000000718204090B0B0B0B09090C0322D
:100300000D0000F0FCFEFFFFFFFFFFFFFFFFFEFC04
:10031000F00000071F3F7FFFFFFFFFFFFFFFFF3FD2
:100320000D00E01008C40202020202020202C40828
:10033000F0000708182C535754B7B7B4978380F0D0
:100340000F00E0F0F8FCFEFEFEFEFEFEFEFEFCF8F6
:10035000F000070F1F3F7F7F7FFFFFFFFFFFFFFFC3
:100360000F00E01008040202020202020202040866
:10037000F000070818204346545454545643403064
:100380000F00E0F0F8FCFEFEFEFEFEFEFEFEFCF8B6
:10039000F000070F1F3F7F7F7F7F7F7F7F7F7F3F43
:1003A0000F00000400000401020500030600220102
:1003B0001001FE00EE00DE00D600C800BA00AC005E
:1003C000180E1400070E130013080500020E121277
:1003D000000A0518FF180E1400070E13000100088C
:1003E00005011113FF740162014B01180E1400077F
:1003F0000E13001308050012160E1104FF180E1438
:1004000000070E130001000A0518FF010201010197
:1004100003030202011010FFFFFFFFFFFFFFFFFFBA
:10042000FFFFFFFFFFFFFFFFFFFFFFFFFFFFFFFFDC
:10043000FFFFFFFFFFFFFF00FCA2428242C24242D9
:100440003C003C72423C8000316AEB8A8A7380FF38
:10045000FFFFFFFFFFFFFF00FCA252A2C2FC01FF53
:10046000FFFFFFFFFFFFFF00315A6B59687086FFE7
:10047000FFFFFFFFFFFFFFFFFFFFFFFFFFFFFFFF8C
:10048000FFFFFFFFFFFFFF017C6A526A5262444494
:100490007C017C6242643D8EB1B1293E80BFA834AC
:1004A000793E00FFD13E800379542A562990C8D363
:1004B0009C003E5264780300EEAAEEEEEEEEEEEE05
:1004C000EEEEEEEEAAEE0000775577777777777746
:1004D0007777777755770040001000000101000022
:1004E00000000404000040800808404002020010A0
:1004F000100000040400800AEEEE0E060606060652
:100500000606060EEEEE0A20BFBFE0C0C0C0C0C0A7
:10051000C0C0C0E0BFBF20FFFFFFFFFDFBFDFFFF2E
:10052000FF7FBF7FFFFFFFFFFFF7EBF7FFFFFFFF3F
:10053000FFFFFEFFFFDFFF00000000240027002A6E
:10054000002D00300000000000250028002B002EA8
:10055000003100040802011040804010204080401B
:100560008008020401804020100201108010204009
:1005700040200404040404030405020202020403EC
:10058000020202020606060606060404020202042D
:100590000406011501260137014A015D0172018837
:1005A000019F01B801D201EE010B022A024B026E3B
:1005B000029302BA02E40210033F037003A403DCB7
:1005C00003170455049704DD0427057505C80520A5
:1005D000067D06E0064907B8072D08A9082D09B9C8
:1005E000094D0AEA0A900B400CFA0CC00D910E6FEF
:1005F0000F5A1053115B1272139A14D415201780DE
:1006000018F519801B231DDE1EB420A622B524E494
:10061000263429A72B402E0031EA330037453ABC57
:100620003D68414C456B49C84D68524F57805C004E
:100630006210111213151617181A1C1D1F212325DD
:1006400027292C2E3134373A3E4145494E52575CCA
:1006500062686E757B838B939CA5AFB9C4D0DCE9CF
:10066000F7D5F08D14A1C881CFD9F1AF2000030ECA
:100670000D0711011312FF90270028911D002880FB
:1006800000288190270028911D0028800028819053
:10069000270028911D00288000288190270028919C
:1006A0001D00288081F0906D000F80F09045001EA5
:1006B00080F0901D006480F0EEFCFE000BFC020058
:1006C000FBEC00FEFF0600020000000100FF01003D
:1006D000FF00010000001008007E424242424242F8
:1006E0004242424242427E00081000FE02020202E2
:1006F000FE00007F404040407F00080800000000EE
:10070000000000008142001818004281FF0402101E
:10071000140913FF07010C05000E150511FF100841
:10072000FFD5ABD5FF001F1F1818FFFF0003FFFF09
:10073000030800000007050707070704050B05135A
:10074000050012011505FF120617FF12061719FF03
:100750000D05160007010C05FF030E0D13090D14FE
:1007600005FF0918387CEEC783C7EE7C38FC000013
:10077000FF01FF0000FCD8F870FFACFF000003375A
:1007800010F80C0CFCFCF000FCFC0C0CFCFCF8F071
:1007900000FCFC0C0CFCFCF8F0003CFC8080FCFC39
:1007A000FC3C00FCFCFCF8E080E0C3070EFC18FCFD
:1007B0000E07C3000CFCFCF03F06063F3F3F003F26
:1007C0003F06063F3F3F3D003F3F30303F3F1F0F5A
:1007D0000000013F3F3F3F0100003F3F3F00030F4C
:1007E0001F8F0000FFC0FF00003F06063F3F3F068F
:1007F00008002640402600FFFFFFFFFFFF0608001D
:100800000670700600FFFFFFFFFFFF0608000000F4
:100810000000000F9AF1F11A0F03080000006E7A31
:100820000E0708000C1C381C0C000C1E3E7C3E1EE3
:100830000C0708001800000000003C7E7EC3C36661
:100840003C0808000008000000000000387C7E7DA5
:100850003900000808007C7E0E060606007CFEFFBC
:100860007F0F0F0F060608002640402600FFFFFFFF
:10087000FFFFFF0608000670700600FFFFFFFFFF86
:10088000FF0708000C1C381C0C000C1E3E7C3E1E92
:100890000C0708001800000000003C7E7EC3C36601
:1008A0003C0808007C7E0E060606007CFEFF7F0FDB
:1008B0000F0F0606100000FEFE00000000030300FC
:1008C0000000FEFFFFFE0004477F7F47040808E3A7
:1008D0008D121212128DE3E38D1E1E1E1E8DE30873
:1008E00008E3CD90969690CDE30808E00E2E203DCB
:1008F0000101011010013EB22A9C009E3C3002060C
:10090000E09CC23C81807F536C30010205000000F6
:100910003C566A7C810E10F1ED9D7BF7F7EFEFF707
:10092000F77B9D6DF18FB7B9DEEFAF37B7EFEFDE35
:10093000B9B68E0808C3BD66424266BDC31010FF3B
:100940000180C6E7F73B3D3D3BF7E7C68001FFFF6F
:10095000FCFBF7EFDFB67070BEDFEFF7FBFCFF10BC
:1009600010FFFF07031303C3C3C3C303130307FF2E
:10097000FFFFFFE0C0C8C0C2C3C3C0C0C8C0E0FF23
:10098000FF101000F82442F181E1F1E10135190274
:1009900004F8000000013E60D9999D86869A9CE08B
:1009A000100F0000F8FCFEFFFFFFFFFFFFFFFFFE40
:1009B000FCF8000000013F7FFFFFFFFFFFFFFFFF8C
:1009C0001F0F0000F04884E202C2E2C2026A320451
:1009D00008F00000011AE499839B9B9D9C9C8098E1
:1009E000D8271800F0F8FCFEFEFEFEFEFEFEFEFC20
:1009F000F8F00000011BFFFFFFFFFFFFFFFFFFFFFD
:100A0000FF3F1800E01864020202020202020264C0
:100A100018E0000007788890B0B0B0B0B09090C0F7
:100A2000320D0000E0F8FCFEFEFEFEFEFEFEFEFCC7
:100A3000F8E00000077FFFFFFFFFFFFFFFFFFFFF62
:100A40003F0D00F008046281810181810181816292
:100A500004F8000F106C86919B9ABBBBA29B99EE89
:100A6000100F00F0F8FCFEFFFFFFFFFFFFFFFFFE8F
:100A7000FCF8000F1F7FFFFFFFFFFFFFFFFFFFFFDF
:100A80001F0F00F04884E202C2E2C2026A32040888
:100A9000F00000252644419B839B9D9C9C98809858
:100AA0005B2418F0F8FCFEFEFEFEFEFEFEFEFCF8E7
:100AB000F000003D3F7F7FFFFFFFFFFFFFFFFFFFD5
:100AC0007F3C1800F00C32010101010101010132EB
:100AD0000CF000000718204090B0B0B0B09090C06B
:100AE000320D0000F0FCFEFFFFFFFFFFFFFFFFFEE7
:100AF000FCF00000071F3F7FFFFFFFFFFFFFFFFF2E
:100B00003F0D00E01008C40202020202020202C409
:100B100008F0000708182C535754B7B7B4978380D0
:100B2000F00F00E0F0F8FCFEFEFEFEFEFEFEFEFC16
:100B3000F8F000070F1F3F7F7F7FFFFFFFFFFFFFE2
:100B4000FF0F00E010080402020202020202020487
:100B500008F00007081820434654545454564340A4
:100B6000300F00E0F0F8FCFEFEFEFEFEFEFEFEFC96
:100B7000F8F000070F1F3F7F7F7F7F7F7F7F7F7FA2
:100B80003F0F000F100000E0F038FCFC3CFCFCD8EC
:100B9000F0E00000001C372F3E3F3F3E3F3F3F3F0D
:100BA0002F3C0000E0F0F8FCFEFEFEFEFEFCF8F03C
:100BB000E0003C7F7F7F7F7F7F7F7F7F7F7F7F7FA6
:100BC0003C10100000E0FCF0E0F890F098E0F0FC41
:100BD000E0000000001F7F3F0F0F1F1F0F0F3F7F20
:100BE0000F000000E0FCFEFCF8FCF8F8FCF8FCFE4E
:100BF000FCE000001F7FFF7F3F1F3F3F1F3F7FFF45
:100C00007F0F0000F0E0C080E0F890F098E080C036
:100C1000E0F000000F0707070F0F1F1F0F0F070758
:100C2000070F00F0F8F0E0E0F8FCF8F8FCF8E0E07E
:100C3000F0F8F03F1F0F0F0F1F1F3F3F1F1F0F0F39
:100C40000F1F3F0E08003070606060607078647C39
:100C50006438003078F8F0F0F0F0F8FCFEFEFE7C2E
:100C600038000030786078607C727E723C00000052
:100C700030F8FCF8FCFCFEFFFFFF7E3C000808DBC0
:100C80009924DBDB2499DB0D10008000003CE66634
:100C9000FE5EE63C000000032B0900101414006007
:100CA00044060080C0E0FCFEFFFFFFFFFFFEFC806B
:100CB000077F7F7F3F3F3F3F7FFFFF4F0F080800C9
:100CC00000000000000000381C163838161C3800E0
:100CD000000000000000000070BC3838BC70000844
:100CE00008003C667E667E3C003C7EFFFFFFFF7E88
:100CF0003C007848784878780078FCFCFCFCFCFCE8
:100D00007803080000006E7A0E0708000C1C381CDF
:100D10000C000C1E3E7C3E1E0C0C08E18E080838B0
:100D200048483808088EE1C09E1212727272721220
:100D3000129EC00808000008000000000000387C77
:100D40007E7D3900000808007C7E0E060606007CC9
:100D5000FEFF7F0F0F0F060F1000000080808080C5
:100D600080808080808080000000000101010101FE
:100D700001010101010100000080C0C0C0C0C0C06D
:100D8000C0C0C0C0C0E000000103030303030303AD
:100D90000303030307000000000000FEFE00000044
:100DA0000000000000000000000007070000000035
:100DB0000000000000000001FFFFFFFF0100000035
:100DC00000000000000000070F0F070000000000F7
:100DD00000EA0D530841083108210819080B08FDE5
:100DE00007EF070508FFC1D5EBFF06100000FEFE68
:100DF000000000000303000000FEFFFFFE000447A8
:100E00007F7F4704051014090FFF03080000000747
:100E100005070707070C010FFF0308030603040477
:100E20000406080000000000000F9AF1F11A0F08F4
:100E300008000008000000000000387C7E7D3900BA
:100E40000003080000006E7A0E0508FFC1D5EBFF15
:100E5000B308A1082F0E91088108410E210E7308D6
:100E60006508570D041B0000450DC40DA70D330D7B
:100E7000520E0000190DE9100000090D00000000DD
:100E8000010D00000000DF0CB4100210BD0C48156D
:100E90000811870C001E02107D0C451BDA1E430C46
:100EA000431F0210C10B48150811830BD314021005
:100EB00081091514D90F0000000000005F0900002F
:100EC000670E3D090000670E3309F41E0000150986
:100ED000930D0000F3080000CF1F00001D21EB1A46
:100EE000E90800009720DF080000841B00000000D4
:100EF0000000CD08FC1A2820080B000202020100A5
:100F0000090400000102020000052400100105246C
:100F100001010104240206052406000107058103DE
:100F200010004009040100020A0000000705020247
:100F30004000000705830240000004030904120179
:100F40000002EF020140412336800001010203014B
:100F500041726475696E6F204C4C43004172647538
:100F6000696E6F204C656F6E6172646F000305A53A
:100F7000096C0962010FC403165206690FC80415F3
:100F80008BB5841544156B042E6F130416B91639EE
:100F9000038A680A6B0A490306C906CBA3A6050E95
:100FA0006FA324152B1748169C0302440494CE6F9C
:100FB0000413080776073607B605B62516451685C5
:100FC0000829086C0503A703870327D7CB0347032A
:100FD0002346340815A4020FC80679030FC8066813
:100FE000068803B6270A6D0A42020665AE6F034AF9
:100FF000280AA50AC80615B415B91579A4CB0AABF9
:101000000A5B050F040F6C0FC40F2C0FAC033408E0
:1010100034D42C29078822882D8A63867D8A668AA3
:101020004A884D0516C5076207A547C9070F01166F
:1010300029028E2F83A6040F040778078A076B0501
:1010400043270952095C0972097C040A270AA70A86
:10105000C90A48010F60030FC80A230A5D054E6FD5
:1010600068226842688268A207146E146007B62777
:101070003607B9072907CB030F600AAB0A2C011307
:10108000C4053404183CF8ACB6A508CC050F6D16A1
:10109000251629072D07460388250A2806B50215B7
:1010A000C51729020FC4086904036503A50325D7E2
:1010B0001A031061563756A7021388A3A5040FC858
:1010C00008690859082A026E6063A7044729486521
:1010D000484D4657041060174917281542022DA5A0
:1010E00034040110C5032C653404146F01834502D8
:1010F0000A560A4901A363012B2504146F2B6417B8
:10110000A8172803832417641548061460146F2A4F
:10111000A92A252A492A8B021833A38805EE6F18BD
:10112000A9340834D4153B0318350A430A1703348D
:1011300048F826186D06E942E94CE952E95CE97283
:10114000E97C041308064506650685070F08168422
:101150000733076D074707B2077303162A16340FC4
:101160006C02089908790408280848086C088C055E
:101170002E8007CB0785079C07A503063B067B0649
:101180005B0213A4CEA4020AAB0A59020569A62386
:1011900001082903079607B907D602065706790200
:1011A000A625A637010F040183470213808E800312
:1011B00017891557AE20040367038703A7D72904AF
:1011C000A61615491569158901138C02087A084974
:1011D00002034504C501A66504F85414646E60F862
:1011E00084021364EE64020AB50A49020FC8086556
:1011F00003066406760667000217681583010EA4CD
:1012000003064906690689010639010F88018385AD
:10121000020A540A850213244E249E0F970F900F42
:10122000870F7E0F770F740F6D0FE20FDB0FD60F56
:10123000CF0FC40FB90FB00FA90F2E102310141029
:101240000D100210F50FEE0FE90F68105D1056102B
:1012500053104A103F1036103110A810A3109E10E2
:1012600097108C1081107E107710E210DD10D410D2
:10127000CB10C610BD10B810B1100A110311FA102E
:10128000F710F410EF10EC10E5105A114B11421149
:1012900035112E1127111C1117118B118611811177
:1012A0007A116F11661161119F119A11F711F711DF
:1012B000F71193119011BF11F711B611AF11AA11C7
:1012C000A711A411D811F711D511D011F711CB1115
:1012D000C811F811F711F011EB11F711E611E11136
:1012E000151210120D120A1207120012FD1190278A
:1012F00000C89131060081006480F00102000703FC
:1013000007060004050600000200000303020506AC
:101310000104038A127A126A125A124A123A122AE3
:10132000121A122703080800000B0014001B0025E6
:101330000033003F004C00540060006E00780082D3
:10134000008E009B00A400AF00BA00C400CF00D9FB
:1013500000E400EE00FA00060111011A0126013036
:10136000013B0145014D01580164016F0179018381
:10137000018F019901A501B001BA01C301CD01DAC4
:1013800001E501ED01F90103020C0216021B02271F
:101390000231023B024802530260026C0275027E77
:1013A000028702900298021F1B92F10C2F204440EA
:1013B00044401F1B42F104F308F134F54F104F2055
:1013C000F3404F1B4F204F2044F0304044466444CC
:1013D0000466404F0046404004004BB6BB400060EE
:1013E00004F06F2060044BBB4B4404F2040404433C
:1013F0004044404BF14F2044F10F4444109444F1D9
:101400000444F00F040A441BB64442006000200666
:1014100000F04644401F1B9F20CF36833033A01F6F
:101420000B042F202F208F030440400400040040B1
:1014300000F0404F230006009000600C0006566F3D
:1014400020404BBBF04F204000F6401F1B9F20C2A6
:10145000F10C833033A044404442F202F10C8F136C
:10146000A01F1B9F20C2F10C8F13A01BB0BB92F1D9
:101470000CF36200060CF14044F1044F1044F134C7
:101480001BB0BB92F10C2F10C8F13A2F1042F1049F
:101490002F204F1040F046BF040604F0050F1463E0
:1014A000404440F04F1042F10C444044401F1B9216
:1014B000F202F10C444044401F1B9F302F10C8F132
:1014C0003A200060CF0060CF160C8F0304F362F166
:1014D0000C2F10C833033A1F1B42F202F104833071
:1014E00033401F104F20C2F10C8F13A0F840444F1F
:1014F0000044F1044440444F20C4F10C4F13A01B9E
:10150000B0BB92F10C2F10C833033A1F1B92F10CA1
:101510002F10C833033A1F0B042F1042F208F13A80
:101520004440F240444F20C8F13A1BB0BB92F10C4A
:101530002F10C40444044F1B42F202F1044F134025
:101540004F104006660C406660C4F10C44F1644FD5
:101550000064F10640F1401BB0BBB2F202F208F1A8
:101560003AF2B9F20CF20C8F10C01F1B92F10C2F43
:10157000208F13A01BB6BB42005F20500C83363374
:10158000404044404F304F1044040404F34F20C8FF
:10159000F10CF3404F10C204440C204040C8F10C41
:1015A000444BF240F240F24044401F1B92F202F2E0
:1015B00008F13A1F10CF20CF3020006660FA4F307C
:1015C000F3404BB6BB42006004000600F4404040CC
:1015D0004042F10C2F10CF341F1B42F1042F204446
:1015E000F0344F10C440404C400400C48F00401FF2
:1015F0001B92F10C2F10C833033A1B6F0B206F00A6
:10160000206F0083603330F00666F0060CF0050CA6
:10161000F0353A44F0B44F204F10F440F44F204FCF
:1016200010F04044401F1B9F304F204F134044F0A8
:10163000B4F20404F10F344BF0044F8044F1344F02
:101640001B4F2044F00444F0344003070007040219
:1016500001040600070407050706E012D212C412AF
:10166000B612A8129A12BE01070600000A00130063
:101670001C0025002B0030003D0045004F005300AA
:101680005A0064006C0074007D00830088009200A2
:1016900098009E00A800B000B400BD00C600D400B1
:1016A000DC00E900F200F700FD00070110011B015A
:1016B00026012E01370141014A0153015C01444FCB
:1016C00006444F062F202F2066F1B66F206F206F43
:1016D00010BB4F0B004F20F14F30F2B4F20F140447
:1016E0004F2040FB4F204F1040FA4F304F26446FA1
:1016F00014060474005000CF0644402F202F20F31E
:1017000068F23006F206F1066F103F1040FF000F3E
:1017100034F204F204F30F344F10F14F104400047C
:10172000F2004F26F206F206F204F46F4400F14094
:1017300004444447F04F204F20F3404F104FA04F38
:1017400020F34FC0F1404BBB444F104F2040F340BB
:101750004FF0040F0400F204F9040F244400444F36
:1017600020440040F540F341F202F202F2004FF053
:10177000F40000F14004F204F20F1447F14F006F3F
:1017800020600F3440F0400040040004004044401A
:1017900004400F2404F20400F640F0404400040426
:1017A00044F0044400F0402F202F202F202F104021
:1017B000FF0004F20000F14FD0F040F34F1044F16D
:1017C0000444F0044044400444F204F20F34F34F64
:1017D00000666F006664000444400F1400F1400F7F
:1017E0001400F0402F104F362F104F364F2066F167
:1017F000046F10F360000F04000F04F204F3604F55
:1018000000444F204F20F360F04744F204F204F309
:10181000604000F04F204F20F360400F04000F04A1
:10182000F1044F3601020408102040800F0F0F0F03
:10183000F0F0F0F004080FAFAF0F006464610046F1
:101840004669006A6A2E600B6BF0007D7A7600DED6
:10185000BC0000A6A68000A62280E404E2E2807715
:10186000778060979360D8B3DBE8FF0114017700BD
:10187000140177009601D70014006700B401270017
:1018800000017721000177110001FF21000177019C
:101890000B00C7110B01FF810A01EF610A0177F00C
:1018A0001E01F3000000FF100000FF10000077028F
:1018B0001400FF011400FF100000F700140077006F
:1018C00000007700000000000000771000001010FA
:1018D00000F82442F181E1F1E10135190204F80038
:1018E0000000013E60D9999D86869A9CE0100F0009
:1018F00000F8FCFEFFFFFFFFFFFFFFFFFEFCF8000C
:101900000000013F7FFFFFFFFFFFFFFFFF1F0F00F2
:1019100000F04884E202C2E2C2026A320408F00027
:1019200000011AE499839B9B9D9C9C8098D8271862
:1019300000F0F8FCFEFEFEFEFEFEFEFEFCF8F000EF
:1019400000011BFFFFFFFFFFFFFFFFFFFFFF3F182F
:1019500000E0186402020202020202026418E000BF
:101960000007788890B0B0B0B0B09090C0320D0051
:1019700000E0F8FCFEFEFEFEFEFEFEFEFCF8E000CF
:1019800000077FFFFFFFFFFFFFFFFFFFFF3F0D008F
:10199000F008046281810181810181816204F80083
:1019A0000F106C86919B9ABBBBA29B99EE100F0007
:1019B000F0F8FCFEFFFFFFFFFFFFFFFFFEFCF8005B
:1019C0000F1F7FFFFFFFFFFFFFFFFFFFFF1F0F0046
:1019D000F04884E202C2E2C2026A320408F0000067
:1019E000252644419B839B9D9C9C9880985B241852
:1019F000F0F8FCFEFEFEFEFEFEFEFEFCF8F000002F
:101A00003D3F7F7FFFFFFFFFFFFFFFFFFF7F3C1892
:101A100000F00C320101010101010101320CF00062
:101A2000000718204090B0B0B0B09090C0320D00C8
:101A300000F0FCFEFFFFFFFFFFFFFFFFFEFCF000DA
:101A400000071F3F7FFFFFFFFFFFFFFFFF3F0D006E
:101A5000E01008C40202020202020202C408F000FE
:101A60000708182C535754B7B7B4978380F00F006A
:101A7000E0F0F8FCFEFEFEFEFEFEFEFEFCF8F000CE
:101A8000070F1F3F7F7F7FFFFFFFFFFFFFFF0F005D
:101A9000E010080402020202020202020408F0003E
:101AA00007081820434654545454564340300F00FE
:101AB000E0F0F8FCFEFEFEFEFEFEFEFEFCF8F0008E
:101AC000070F1F3F7F7F7F7F7F7F7F7F7F3F0F00DD
:101AD000733511241FBECFEFDAE0DEBFCDBF11E0BA
:101AE000A0E0B1E0ECE5FFE602C005900D92A8345D
:101AF000B107D9F727E0A8E4B1E001C01D92A73FE4
:101B0000B207E1F71DE0C9E6DDE004C02197FE0160
:101B10000E94A137C836D107C9F70E9411330C942F
:101B2000AC370C940000FC018689843119F490894B
:101B30009B5F908B418F178A882329F08150868B79
:101B40004370408F02C08FEF86838FEF0895CF934D
:101B5000DF93FC01DA01EB019E818EEF890F843067
:101B600058F4933049F0ED91FC910480F581E02D1B
:101B7000CA01DF91CF9109949650983008F4168AE3
:101B80008FEFDF91CF910895EF92FF920F931F9304
:101B9000CF93DF93EC01FB01042FE780F0841185E4
:101BA0008E89843151F02F8138858985082E000C6B
:101BB000990B4E8941111CC02EC08189898BF886F2
:101BC000EF828AEF810F898787E796E00E943D24A4
:101BD00080919F06853039F7E6EAF6E0808185310D
:101BE00009F4128A7D9687E0EE38F807B9F7DBCF63
:101BF00041504E8B4989413059F02CF4411135C088
:101C00002350310932C0423051F1433069F12DC0C7
:101C10002D5F3F4F2AC0412F110F550BB701621B9B
:101C2000730B6E5F7F4F6530710558F4BA01681B06
:101C3000790B6E5F7F4F6530710518F44FEF4E835F
:101C400014C0E216F3061CF42350310905C02E150A
:101C50003F0514F42D5F3F4F4817590714F40397BD
:101C600004C0841795070CF4039638872F8389875F
:101C7000023370F4083240F40E3140F4043140F481
:101C800081E00A3030F402C081E003C080E001C08E
:101C900083E0888F8FEFDF91CF911F910F91FF909D
:101CA000EF900895FC018489882349F0968999234F
:101CB00041F09150968B9B3311F48CE3818F8FEF21
:101CC000089587E796E00E943D2482E10895CF932E
:101CD000DF93FB0126812E3F09F5EC018E818F30C9
:101CE00059F4E091C501F0E0E854FE4F83811816E5
:101CF000ACF4815083830AC0803181F4E091C50146
:101D0000F0E0E854FE4F8085181644F40E94FD234D
:101D10008FEF8E838CEA96E00E943D248FEFDF9157
:101D2000CF9108950F931F93CF93DF93EC018B0115
:101D3000FB018681833009F0A6C08A859B85988740
:101D40008F832C8529878185082E000C990B079697
:101D5000022E000C330B821793070CF024C18789E5
:101D6000811121C181E0878B8CE38AA387818E5FFB
:101D70008D8F81858A508E8F8F8D98A1FC01E457BD
:101D8000FF4F2081263009F5379685589E4F30E069
:101D900040E020E05081533081F4618951E06130AE
:101DA00021F050E0211107C002C02111DAC021E06A
:101DB000613009F420E04F5F350F7D968E179F0745
:101DC00049F74313C7C085E002C0FB0184898BA398
:101DD0008BA1823031F493E0FE01E15AFF4F9083F2
:101DE00008C0811106C091E09093B9010BEE13E099
:101DF00002C000E010E09FEF980F933090F49091B4
:101E0000BA019F5F9093BA01FE01E25AFF4F8083AF
:101E1000E82FF0E0EE0FFF1FED51FC4F05911491FC
:101E200018C0843049F48091B8018F5F8093B80165
:101E30008C8B05ED13E019C0853059F4E091C50194
:101E4000F0E0E854FE4F83818F5F83830DEF13E052
:101E50000CC0863051F4E091C501F0E0E854FE4F2B
:101E600080858F5F808700EC13E08AE891E00E9414
:101E70003D240E94FD238F8D98A1FC01E657FF4F62
:101E80001183008363C0FB018589882389F0898DD4
:101E900081110EC08C8981508C8BAB01BE01CE01AB
:101EA0000E94CE2E8AE991E00E943D248EE1898F26
:101EB000F80186818430A9F48FEF86838C89082EFF
:101EC000000C990B2091B801022E000C330B0196E7
:101ED000281739070CF4C9018C8B8CEA96E00E9414
:101EE0003D24F8018681823099F48FEF8683FE01CC
:101EF000E15AFF4F8081282F30E02430310514F45F
:101F00008D5F01C086E080838CEA96E00E943D24CC
:101F1000F8018681853009F046C08FEF8683E09115
:101F2000C501F0E0E854FE4F83818F5F83830E94F8
:101F3000FD238AE891E00E943D248F8D98A1FC0149
:101F4000E657FF4F2DEF33E031832083319722E8AE
:101F5000208329C08AE891E00E943D2488E08BA379
:101F600022C087E08BA38AE991E00E943D248C89FE
:101F70001816BCF481508C8BA801BE01CE010E94C2
:101F8000CE2E8F8D98A1FC01ED56FF4F85589E4FA8
:101F90002081233009F4118A7D968E179F07C1F79F
:101FA00002C080E0E8CF8FEFDF91CF911F910F91BA
:101FB0000895CF93DF93EC01FB018681813131F4E9
:101FC00084E68E8B84E08093000118C0811116C0D6
:101FD00080910001843091F4898D81110FC08C892A
:101FE00081508C8B84E6898FCE010E94CE2E8C8905
:101FF000811104C08FEF8E838093FA058FEFDF91FC
:10200000CF910895CF93DF93EC01FB01868182315C
:1020100031F09E819C30E1F095891916CCF4998DB0
:10202000911116C08C89FB019589891B8C8B181620
:102030004CF08E818C3011F40E94FD238FEF8E8343
:102040008DEF0BC0CE010E94CE2E84E1898F04C09B
:10205000813011F484E68A8F8FEFDF91CF9108955C
:10206000EF920F931F93CF93DF93EC01262F898D6F
:10207000882331F063E00E946D37913009F46EC01F
:10208000822F9AA1992339F1EBA1F0E0EE0FFF1F07
:10209000E255FC4F45915491EE24E3948091C501A3
:1020A000811101C0E12C6E8D062E000C770B9695E8
:1020B0009695969526E030E0F901E91BF1096E1B33
:1020C0007F0B8D8D00E020E0082E000C990B0E9404
:1020D0006E2F22E035C09AA549A1992349F0FE014F
:1020E000E95BFF4F90819F7E913021F4942703C0DC
:1020F00091E001C090E03989E32F032E000CFF0B23
:102100008F01000F111FE00FF11FE90FF11DEE55B8
:10211000FC4F2491911103C002E010E002C001E0E5
:1021200010E0E00FF11F0491442351F066E00E949B
:102130006D3780FD05C0323010F42F5F01C001E023
:102140006985062E000C770B685071098F81988580
:10215000E12C40EA51E004970E946E2FDF91CF916D
:102160001F910F91EF900895CF92DF92EF92FF921F
:102170000F931F93CF93DF93EC018B01C42E0E942A
:102180009D36D12CE12CF12C2DE330E040E050E0E5
:102190000E940A37C616D706E806F90641F4B801C8
:1021A000CE010E943C2F81E08F8B8AE08E8B8E893E
:1021B000882329F081508E8B811101C01F8A8FEFF7
:1021C000DF91CF911F910F91FF90EF90DF90CF9013
:1021D00008950F931F93CF93DF93FC012689243139
:1021E00089F48B01EC01168A0E94EB20882351F0C0
:1021F000F8018781908598878F8381859889891BCD
:10220000815089878FEFDF91CF911F910F910895B2
:10221000CF93DF93EC01FB018589968118161CF0A2
:102220009130E9F402C0913009F4168ABF018C891B
:1022300081508C8B81110EC08E818B3039F46FEF01
:1022400083E196E00E94F11F0E94FD238FEF8E83B1
:102250008DEF06C0CE010E94CE2E84E1898F8FEFD4
:10226000DF91CF9108952F923F924F925F926F929C
:102270007F928F929F92AF92BF92CF92DF92EF9216
:10228000FF920F931F93CF93DF93CDB7DEB72B97BA
:102290000FB6F894DEBF0FBECDBF1901A986411558
:1022A000510509F4D2C11FEF811611F0712C01C044
:1022B0007E2CFA01F4903196E491AF2DB0E04D01FF
:1022C000880E991E181419040CF0BFC180389105AE
:1022D0000CF0BBC1A62E062E000CBB0895012E0FDC
:1022E000311D121613060CF0B0C160340CF0ADC1F4
:1022F0004E5F5F4F01111A01DE2ED694D694D6940C
:10230000E77071E009F470E0272F30E02D0D311DEA
:102310002A9FF0012B9FF00D3A9FF00D1124EE2023
:10232000C1F07E9E20017F9E500C11249101240D4E
:10233000351D38872F83EE9E3001EF9E700C1124DF
:10234000460D571D002381F0240D351D460D571DE8
:1023500003C0002339F0910189010E0F1F1F188758
:102360000F8302C038862F82F501B7FE03C0F195B6
:10237000E195F1091E2F1770712E062F67FF02C01D
:1023800007E0060F05950595059567FF06C07720C0
:1023900021F00150E8E0E7197E2E97FF05C0EE27F7
:1023A000FF27E81BF90B02C0E0E0F0E020E882160E
:1023B000910424F010E8612E681A01C06F2C6E1A87
:1023C000A02E002E000CBB080F3F1CF4EA2CE0945A
:1023D00001C0E12CD70EAD0CB11C39E0A316B1043D
:1023E0001CF018E0D12ED01ADE18902E9E0C892CED
:1023F0008C01792D20E87203000D111D11240E0FA0
:102400001F1FFE9C70011124EE0DFF1D4E0F5F1F5C
:102410002F8138852E0F3F1F7C2D71707D83C0FE6C
:1024200014C0A62CB12CF50131974E0F5F1F2E0F53
:102430003F1FFD01EA19FB0997FF03C0F195E195E4
:10244000F1094E0F5F1F2E0F3F1F8C2D82708E8360
:10245000C1FE17C08D2D90E001978A9FF0018B9FE0
:10246000F00D9A9FF00D11244E0F5F1F2E0F3F1F8E
:1024700067FF07C0F194E194F1084E0D5F1D2E0D2A
:102480003F1D81E090E02C01072C02C0440C551C3C
:102490000A94E2F7CD01880F991F66277727681BFA
:1024A000790B78876F830C501E4F9D0C862D90E022
:1024B0006D01C81AD90ABC016A0F7B1F7B876A8726
:1024C000891409F4C2C0580170E8A70EB11C750147
:1024D000B0E06B1609F49FC0FA01A49121143104F5
:1024E00021F0F901849190E002C08FEF90E06985BE
:1024F000662311F0A095A8237E817723E9F1A295A8
:10250000EA2FEC7CE695E695A373F4E0AF9FB0016B
:1025100011246E2BA62FAA7A7A2F76956575A62F91
:10252000AA0FA72BBC01E4E076956795EA95E1F741
:10253000F4E0880F991FFA95E1F79927682B792B1A
:10254000CB018C7C9927FC01F695E795F695E795EC
:10255000CB0183739927880F991F880F991F8E2BA2
:102560009F2BBC016A7A77277695679585759927A1
:10257000880F991F862B972B9C838B83A49DB0017A
:10258000A59D700D11247A836983EB81FC814E9E99
:10259000C0014F9E900D5E9E900D112480959095E8
:1025A0009C838B83E985E23081F487FC04C0F801C9
:1025B0008081682760837720D9F0F6E0F815C4F0B1
:1025C000F70190818A81892712C087FC05C0F80134
:1025D00090818923682B6083772051F0F6E0F8150D
:1025E0003CF0F70190818C8189239A81892B80832B
:1025F0006D81662329F0415051092150310904C0F1
:102600004F5F5F4F2F5F3F4FBF5F7FEFE71AF70AC4
:102610000F5F1F4F5ECF83948D81882339F00A8529
:102620001B85400F511F200F311F04C04C0D5D1D35
:102630002C0D3D1D1E81112331F06F817885460FD1
:10264000571F260F371F85013BCF2B960FB6F894E7
:10265000DEBF0FBECDBFDF91CF911F910F91FF90D5
:10266000EF90DF90CF90BF90AF909F908F907F9032
:102670006F905F904F903F902F900895FC01222320
:1026800021F07387628744870EC027813085A28539
:10269000B3858185A217B30719F49485981719F0AB
:1026A0003387228784877087678341878189248560
:1026B000A285B3856A177B0771F4042E000C550BB5
:1026C000022E000C330B4217530761F042175307D9
:1026D00044F083E007C081E06A177B071CF480E0C8
:1026E00001C082E0818B0895CF92DF92EF92FF923A
:1026F0000F931F93CF93DF93EC01898D882311F003
:102700008150898F8AA1882319F081508AA383C0C0
:10271000EF80F8840985002E000C110B0E94191916
:1027200084FF02C00E5F1F4F0E94191987FF02C06D
:10273000025011090E94191985FF03C082E0E81AAE
:10274000F1080E94191986FF03C0E2E0EE0EF11CA9
:1027500088E00E948C2F882381F08091B901882322
:1027600061F08AA58F3F49F460E0CE0184960E9413
:1027700025258CE391E00E943D2484E00E948C2F6B
:10278000882389F1FE01E95BFF4F80818F3F59F576
:102790006E01FEE5CF0ED11CF60160816F3F19F18D
:1027A000623039F4319680818823E9F0815080834A
:1027B00003C0633009F461E1CE018F5B9F4F0E943B
:1027C0002525F6018081823071F481E0FE01EB5A0B
:1027D000FF4F80838F8198853D97918380833296C8
:1027E00089858450808319A28AA58823A1F08F81CE
:1027F00098858E159F0539F48985082E000C990B54
:102800008017910741F081E089A320E0402FB701B4
:10281000CE010E943E138FEFDF91CF911F910F9158
:10282000FF90EF90DF90CF900895CF92DF92EF92DC
:10283000FF920F931F93CF93DF93EC018B01F42E44
:10284000BC0184EF95E00E94D21A80910001823091
:1028500049F48091FA058F3F29F484E080930001C8
:102860008EE18E8B80910001813081F160F08330A8
:10287000B1F1843009F05EC08E8981508E8B811158
:1028800059C083E029C08F2D63E00E946D379130DD
:1028900021F4B801CE010E943C2F8F819885F80168
:1028A00027813085821B930B47968F9708F042C093
:1028B0008985082E000C990B2185821B910927FD23
:1028C000939547968F97B0F581E006C060E084EF5E
:1028D00095E00E94252582E0809300012BC00E9494
:1028E0009D366B017C010E949D3623E330E040E081
:1028F00050E00E940A37162FC701B60125E630E0E6
:1029000040E050E00E940A3720E0412FCE010E94B3
:102910003E130E949D3629E230E040E050E00E94E4
:102920000A37DC01CB014496A11DB11D8A8F898F26
:10293000109200012091FA05188E8A8D811104C031
:1029400090910001943011F487E022C09989913070
:1029500069F01CF4992331F01CC0923071F093306F
:1029600091F017C0211114C084E012C0211101C0E0
:1029700084E08F8B81E0888F0CC0222311F082E0ED
:1029800007C085E005C0222311F083E001C086E086
:102990008F8B8FEFDF91CF911F910F91FF90EF9071
:1029A000DF90CF900895CF92DF92EF92FF920F9336
:1029B0001F93CF93DF93EC016B01842F40FD5CC02C
:1029C00063E00E946D37923009F456C08E898A30D8
:1029D00019F4198A82E08E8BEF80F8840985002E25
:1029E000000C110B8989811104C081E0E81AF108FB
:1029F00003C09FEFE91AF90A8E89823019F4015059
:102A0000110902C00F5F1F4F20E0402FB701CE0118
:102A10000E943E130233110530F09E8985E0891B28
:102A20008E8B81E001C080E0E2E6EE16F10428F032
:102A3000998981E0891B898B81E091E04F815885DC
:102A4000F60127813085421753070CF090E0988FEC
:102A5000882331F08A859B8598878F838C85898729
:102A60000E949D3622E330E040E050E00E940A37A9
:102A7000672B682B692B11F08FEF01C086E0DF9187
:102A8000CF911F910F91FF90EF90DF90CF9008951D
:102A90008F929F92AF92BF92CF92DF92EF92FF926E
:102AA0000F931F93CF93DF93EC018B01E42EFE88ED
:102AB000FF2091F0B984CF80D88448E06B2DC60107
:102AC0000E942C19811108C08E818B3009F04FC0F3
:102AD00081E18B150CF04BC00E949D3623E0822EC5
:102AE000912CA12CB12CA50194010E940A37DC0184
:102AF000CB010197A109B1098D870E949D36A501DF
:102B000094010E940A37DC01CB010197A109B109A8
:102B1000282F8E878D85811104C0211102C081E08C
:102B20008E879F858FE6891B9F81292F19160CF0B0
:102B300021E028172CF4923014F0892F01C081E095
:102B400090E098878F8398898FE3891B9985292F37
:102B500019160CF021E028172CF4923014F0892F6C
:102B600001C081E089878EE18E0D8E8B18C08E2D7D
:102B700065E00E946D37911112C0FA94FE8A4E856D
:102B80004B0D8D85B601680F711D87FD7A9520E08C
:102B9000CE010E943E139F8981E0891B8F8B81E0CB
:102BA000F801478150852F813885421753070CF073
:102BB00080E0888F8E818B3029F4F1E0EF1202C023
:102BC00087E001C08FEFDF91CF911F910F91FF90B0
:102BD000EF90DF90CF90BF90AF909F908F9008952F
:102BE000CF92DF92EF92FF920F931F93CF93DF93D9
:102BF0006C017A018B01C0E0D0E0CE15DF0581F0D9
:102C0000D8016D918D01D601ED91FC910190F0817B
:102C1000E02DC6010995892B11F02196EECF7E019A
:102C2000C701DF91CF911F910F91FF90EF90DF903F
:102C3000CF900895CF92DF92EF92FF921F93CF93A0
:102C4000DF93E82FF0E0E35EFE4F1081E62FF0E027
:102C5000603330F4EF5CF94FE491CE2FD0E006C042
:102C6000EE0FFF1FEF5CFA4FC591D4916E01E12C7E
:102C7000F12C60E074E284EF90E0A70196010E94DD
:102C80000A37BA01A9014150510961097109411579
:102C9000510581E06807710580F060E970ED83E01F
:102CA00090E0A70196010E940A37BA01A90141509C
:102CB00051096109710983E001C081E01130E9F037
:102CC000133091F590919100987F892B809391001A
:102CD00050939900409398001092950010929400A0
:102CE000D0936601C093650181E080936401809177
:102CF000710082608093710017C0909167019111FB
:102D000013C090918100987F892B8093810050930C
:102D10008900409388001092850010928400809171
:102D20006F00826080936F00DF91CF911F91FF90C1
:102D3000EF90DF90CF900895809148010895089515
:102D4000089580E090E008950E94A7373FB7F89477
:102D500080916D0190916E01A0916F01B091700111
:102D600026B5A89B05C02F3F19F00196A11DB11DE6
:102D70003FBFBA2FA92F982F8827820F911DA11D21
:102D8000B11DBC01CD0142E0660F771F881F991F5E
:102D90004A95D1F708951F920F920FB60F92112402
:102DA0002F933F938F939F93AF93BF93809169012C
:102DB00090916A01A0916B01B0916C013091680112
:102DC00023E0230F2D3720F40196A11DB11D05C06E
:102DD00026E8230F0296A11DB11D20936801809360
:102DE000690190936A01A0936B01B0936C0180918B
:102DF0006D0190916E01A0916F01B09170010196EB
:102E0000A11DB11D80936D0190936E01A0936F0180
:102E1000B0937001BF91AF919F918F913F912F918E
:102E20000F900FBE0F901F9018951F920F920FB624
:102E30000F9211248F939F93AF93BF93EF93FF93C0
:102E400080916701882309F449C0809157019091CE
:102E50005801A0915901B0915A01892B8A2B8B2BD3
:102E600051F190915601E0915401F091550180810A
:102E7000892780838091570190915801A091590131
:102E8000B0915A01181619061A061B06A4F580916E
:102E9000570190915801A0915901B0915A010197A1
:102EA000A109B1098093570190935801A09359014A
:102EB000B0935A0120C01092630110926701809173
:102EC0006F008D7F80936F0080915601E0915401D7
:102ED000F09155019081809589230CC08091620109
:102EE000811109C090915601E0915401F091550172
:102EF000808189278083FF91EF91BF91AF919F914E
:102F00008F910F900FBE0F901F901895E82FF0E053
:102F1000E35EFE4F8081813019F0833089F008959F
:102F20008091670181111CC080916F008D7F80931B
:102F30006F0080915601E0915401F09155010CC051
:102F4000109264018091630181110AC08091610136
:102F5000E0915F01F09160019081809589238083E9
:102F60000895CF93DF93D1E0E0914C01F0914D01B2
:102F7000DF011196B0934D01A0934C019491892FDC
:102F8000807FC92FCF70803821F48C2F0E94861744
:102F9000EBCF8039F9F4E0911106F0911206099512
:102FA0008D2780936201E0914C01F0914D01CF019A
:102FB000019690934D0180934C0164918091490159
:102FC000C81790F6C13009F052C0809153018111A9
:102FD000CBCF4DC087FD3AC03296F0934D01E093C0
:102FE0004C01FD01A491B0E0B92B20916501309115
:102FF00066010E945E376C507E4F8F4F9F4F28EEC8
:1030000033E040E050E00E943C3720935B01309376
:103010005C0140935D0150935E0180915B01909152
:103020005C01A0915D01B0915E01892B8A2B8B2BF5
:1030300021F581E090E0A0E0B0E080935B01909307
:103040005C01A0935D01B0935E0117C0803E49F41E
:1030500080914A0190914B0190934D0180934C01D6
:1030600083CF803F09F080CF10924E0106C067FDEC
:103070007BCF8C2F0E941A1677CFDF91CF910895C6
:103080001F920F920FB60F9211242F933F934F93DD
:103090005F936F937F938F939F93AF93BF93EF93C0
:1030A000FF9380916401882341F080916301811135
:1030B00004C080916201882351F180914E018823E0
:1030C00081F180915B0190915C01A0915D01B091D3
:1030D0005E01892B8A2B8B2B21F180915B019091D2
:1030E0005C01A0915D01B0915E010197A109B10958
:1030F00080935B0190935C01A0935D01B0935E01AE
:10310000892B8A2B8B2B69F40E94B1170AC09091EE
:103110006101E0915F01F0916001808189278083E6
:10312000CCCFFF91EF91BF91AF919F918F917F9104
:103130006F915F914F913F912F910F900FBE0F9024
:103140001F90189590914901923009F471C0292F70
:1031500030E0F901E35EFE4F4081F901EF5AFE4F86
:103160008083913031F420915101821302C09093F9
:1031700053019F5F9093490190E0FC01EE58FA4F94
:103180002491FC01ED5AFA4F849130E0220F331F55
:10319000F901EB5BFA4F65917491F901E95CFA4F23
:1031A000A591B4919C91982B9C93413019F0433098
:1031B000D9F0089590916400977F909364001092E5
:1031C000800010928100909181009860909381001E
:1031D000909181009160909381007093550160936C
:1031E000540180935601089590916500977F9093C4
:1031F000650010929000109291009091910098605B
:1032000090939100909191009160909391007093B0
:10321000600160935F01809361018091490188237F
:1032200021F06CE380E00E941A1680E00C9486176F
:1032300008958FB18095807F669B88601C9B846019
:103240000895109248013E983F9808953E9A3F9AFB
:1032500081E080934801089597FD12C067FD10C07A
:1032600050E0840F951F8037910554F4460F511D8F
:1032700067FD5A9581E0403451051CF480E00895C3
:1032800081E00895EF92FF920F931F93CF93DF9306
:1032900020917E0130917F01F901C591D491D9012E
:1032A0001296FD0154913196E4915E9F902D112468
:1032B000FD01A4916A9F800D1124E82EF12CD70105
:1032C000AA0FBB1FFD013496E20FF31F65917491A5
:1032D000E92FF0E08F01000F111F6C5F7F4F600F2F
:1032E000711F3197EE16FF0654F4FD013696E20F7A
:1032F000F31FC591D4910C5F1F4FC00FD11FC61B88
:10330000D70B5C2F550FBCE1B40FA0E0A51708F058
:103310004BC08A2F90E0FC01F595E795E60FF71F6B
:10332000E20FF31FE491DA2FD170A0FFE295EF7066
:10333000EF3079F58C010F5F1F4FF801F595E79598
:10334000E60FF71FE20FF31FC49100FFC295CF7085
:10335000FC013296F595E795E60FF71FE20FF31F94
:10336000E491D11101C0E295EF70F42F8C2F90E021
:103370000396CF2FC41BD0E08C179D073CF0CF2FB6
:10338000D0E0C058DE4FE883FF5FF3CFAD5F4F2F33
:10339000BDCF4B1730F4C42FD0E0C058DE4FE883C8
:1033A0004F5FAF5FF42FF3CFDF91CF911F910F915C
:1033B000FF90EF900895AF92BF92CF92DF92EF927D
:1033C000FF920F931F93CF93DF93C82FD0E0C05885
:1033D000DE4FB12CF12C97E0A92E399181E0830FBB
:1033E000F80E8B2D6A2D0E946D378295807F929505
:1033F000907F4091C501A82FB0E0C92ED12C31118A
:103400002DC0411108C08F2D0E946D37913011F1F0
:1034100020E000E009C020E000E0442329F035501E
:10342000EE24E394333008F4E12C45E154E0BD018F
:10343000C6010E94972FB3948CE1B812CECFDF91D2
:10344000CF911F910F91FF90EF90DF90CF90BF90A1
:10345000AF900895E12C0F2D28E0E7CF383078F0B9
:10346000032F10E008501109000F111FF801E55F4C
:10347000FB4F2491F801E45FFB4F0491CECF232F43
:10348000CBCFEF92FF920F931F93CF93DF9300D098
:10349000CDB7DEB761E580E490E00E94FC3688EBB2
:1034A000E82E81E0F82E01E410E0F70161917F0140
:1034B0001A830983CE0101960E9424240F5F1F4FB7
:1034C0000D37110591F70F900F90DF91CF911F915C
:1034D0000F91FF90EF90089580E490E00E94F43601
:1034E00091E0813509F090E0892F08950F931F93A3
:1034F000CF93DF930E946C1A882379F008EB11E0D8
:10350000C1E4D0E0CE010E94F436F80181938F012E
:103510002196CD37D105B1F72BC082E08093B80159
:103520001092B9011092BA011092C501EBEBF1E0D3
:103530001192148281E0E03CF807D1F7E6ECF1E06B
:1035400084ED91E011928E179F07E1F748EB51E06F
:1035500024E080E090E0FA01E80FF91F148E019654
:1035600088309105C1F72150485F5F4F2111F1CF9D
:10357000DF91CF911F910F910895613091F4FC017B
:10358000EA58FF4F28E23CE13183208332961182D2
:1035900010823A9622EB3BE13183208332961182EE
:1035A00010820895DC0116962C9116972F3F89F012
:1035B0005A962C915A97222321F021505A962C93F7
:1035C00008C0DC011296ED91FC911397309709F039
:1035D00009948FEF0895FB0126812E3F59F4DC01F9
:1035E00054968C91882331F08285938590878783C8
:1035F000848581878FEF0895FC012489211102C001
:103600004170478B8FEF0895FC01DB0117962D91D8
:103610003C91189719968C91199751969C919130DD
:10362000C1F054F4911128C0225131093087278309
:1036300084508187178A1FC0923099F09330E1F44B
:1036400021503109308727838A5F818781E0878B0A
:1036500012C0255F3F4F3087278384508187178AA8
:1036600008C025503109308727838651818781E042
:10367000878B908F01C0108E86898150868B811137
:1036800002C08FEF86838FEF0895FC0140FF3AC0A0
:1036900086898B3019F4168A148A16868489918556
:1036A0008130D9F0823029F1811129C0DB011796D0
:1036B0004D915C9118972781308542175307FCF094
:1036C000285F3F4F24173507D4F081E0848B903278
:1036D00014F08EEF0CC082E00AC02FEF290F2733C1
:1036E00070F022E0248B268512160CF48FEF86876B
:1036F00006C08FEF890F873310F0148A16868685EF
:10370000980F91878FEF0895DC01FB0196819E3F12
:1037100041F48285938590878783848581878FEFA5
:1037200008958FEF992319F09151923040F4169635
:103730008C93169754968C91181614F40895089546
:103740008DEF0895EF920F93E12C00E020E04EE121
:1037500057E06CE170E088E390E00E94972F0F91B2
:10376000EF900895EF920F93CF93DF93EC01E12C4C
:1037700000E020E04FE757E06BE070E083E290E08C
:103780000E94972F20E042E657E067E070E08CE46B
:1037900090E00E94972F0E946C1A811103C040E5AF
:1037A00057E002C049E557E06AE28AE20E94332E00
:1037B00080914801811103C047E457E002C04BE407
:1037C00057E062E38AE20E94332E0E946C1A88233B
:1037D00031F04BE357E06AE38AE20E94332E6881BE
:1037E00088E0689FB0011124665D7F4FE12C00E006
:1037F00022E040E357E082E290E00E94972FDF91C1
:10380000CF910F91EF900895CF93DF93EC0180E873
:103810000E948C2F882311F0188217C080E10E942B
:103820008C2F882319F081E088830FC088E00E94E4
:103830008C2F882351F061E08881813009F460E0A9
:10384000CE01DF91CF910C94CD31DF91CF910895CE
:10385000FF920F931F93CF93DF9300D0CDB7DEB7C6
:103860008C0188E00E948C2F882309F449C0F8015C
:103870008081811117C060E0C8010E94CD318CE9C0
:1038800095E2F801EA58FF4F9183808332961182C6
:1038900010828CE399E23A9691838083329611826A
:1038A00010822EC08230B9F4F801108280E490E0DA
:1038B0009A83898360E0CE0101960E94242481E4EA
:1038C00090E09A83898360E0CE0101960E942424CF
:1038D0000E94761A15C0813099F48091480188239E
:1038E00019F00E94211902C00E9426196091480116
:1038F00082E090E09A838983CE0101960E9424247D
:103900000E946C1A811103C0FF24F39402C082E06C
:10391000F82E80E80E948C2F882361F0F8018081C6
:10392000282F30E02230310514F0815001C080E0B2
:10393000F801808380E10E948C2F882361F0F801D8
:10394000808190E02F2D30E00196281739070CF484
:10395000C901F80180830F900F90DF91CF911F91E3
:103960000F91FF900895CF93DF93EC010E943C29C3
:1039700010928D0710928C0710928E07C459DF4F5A
:103980002881213230F080E490E0AC01421B5109E3
:103990009A01220F422F440F822F869560E2681B06
:1039A00070E0942F969580E4891B90E0DF91CF9191
:1039B0000C94762EEF920F93CF93DF93EC0120E4DB
:1039C00040E860E070E080E090E00E94762E44E104
:1039D00057E064E18AE20E94332E688188E0689FA4
:1039E000B0011124665D7F4FE12C00E022E040E34E
:1039F00057E082E290E00E94972F49E557E06AE2A3
:103A00008AE20E94332E4FE057E062E38AE2DF91C0
:103A1000CF910F91EF900C94332ECF92DF92EF92D3
:103A2000FF920F931F93CF93DF939C01FC01E45906
:103A3000FF4F808181508083803209F08EC03B9798
:103A4000808191818351934119F083E193E102C018
:103A50008AE596E191838083F901ED59FF4F8081DA
:103A600091818350934119F083E093E102C08AE48D
:103A700096E19183808380917E0190917F018352B2
:103A8000934119F043E253E102C046E656E15093F8
:103A90007F0140937E0189010B591F4FF3E14332AF
:103AA0005F0739F4F801808163E00E946D37992344
:103AB00019F04656564179F48091C501811109C02B
:103AC000F80180819BEA899F812D112486958F5F63
:103AD00003C080E001C084E08093C5018091C501EE
:103AE000811102C087E001C088E0E9016901FDE6BB
:103AF000CF0ED11CF6018083F801808180937D0177
:103B00007901F6E6EF0EF11CF701608160937C010C
:103B100040917B010E94421920917B01F701408175
:103B2000F8016081CE010E94B52FF6014081F701B6
:103B30006081F80180810E945E2421E041E269E316
:103B400070E0CE0101960E943E1383E08A8B8FEFD6
:103B50008BA7C85BDF4F88831EC081111CC0F90191
:103B6000EA58FF4FD901A259BF4F8D919D910D90F9
:103B7000BC91A02D80839183A283B3833C96D9010D
:103B8000A658BF4F8D919D910D90BC91A02D808323
:103B90009183A283B383DF91CF911F910F91FF9007
:103BA000EF90DF90CF900895CF93DF93EC018E815B
:103BB0008F3F19F1EC81FD813097F1F0CE0109952D
:103BC0009E819F3F11F49AE09B8F8D3FB1F48091CD
:103BD000BA01823014F4C2E001C0C3E00E949D36F5
:103BE0002C2F30E040E050E00E940A37E62FF0E052
:103BF000E45FF84F849101C08FEFDF91CF9108957A
:103C00001F93CF93DF93EC011091C5011F5F212F0C
:103C100030E0E42FF0E08EE190E0B9010E947937C6
:103C2000CF010E947937892B21F4988D81E0891B7F
:103C3000888F842F65E00E946D37911152C08E8964
:103C4000811123C080E190E0B9010E9479376E8B29
:103C50000E949D3625E030E040E050E00E940A37A7
:103C600070E0660F771FFB01E853F94F859194913F
:103C7000189F802D11248D87FB01E753F94F859103
:103C80009491189F102D11241E878E8981508E8B40
:103C90008F856EE6681B862F6F819D85690F962F35
:103CA00062300CF492E0981724F463301CF462E064
:103CB00001C0682F70E088894EE3481B842F498536
:103CC0009E85490F942F42300CF492E0981724F40B
:103CD00043301CF442E001C0482F20E0CE010E9496
:103CE0003E138FEFDF91CF911F910895EF920F93C5
:103CF0001F93CF93DF93EC018091C501882329F0B6
:103D00008E81873021F011E003C010E001C012E085
:103D10008B8D882381F081508B8F062F01706985F0
:103D2000062E000C770BE12E20E04AEF56E08F8143
:103D300098850E946E2F2E812F3FB1F1898D8111C0
:103D400009C08C8D9985EF81F8854A895B8981113D
:103D500009C021C08150898F63E00E946D37913086
:103D600081F722C02D3021F0A0E0B0E060E003C078
:103D7000ACEFBFEF68EF062E000C770B690F711DDB
:103D800097FD7A95E12E088D2F89CD018E0F9F1F0B
:103D90000E946E2F09C0692F990F770BE12E088DB5
:103DA0002F89CF010E94972FDF91CF911F910F9103
:103DB000EF900895FC0194899130A1F4DB011696EF
:103DC0008C918E3F11F0893069F422E0248B268596
:103DD00012160CF49FEF9687893021F486EA96E05C
:103DE0000E943D248FEF08951F93CF93DF93EC0142
:103DF000DB01142F8E89843161F519966C91199726
:103E00005196EC91519724E0E202C00111249C01EB
:103E10002854394FF901749117964D915C91189778
:103E2000470F511D77FD5A9558874F83FC01E75482
:103E3000F94FE491862F8E0F8987F9013296E4912C
:103E4000ED87F9013396E491EE8787E796E00E94CB
:103E50003D248E8981508E8B9D852F813885290F39
:103E6000311D97FD3A9538872F8329859E85920FBE
:103E70009987198F811102C08FEF8E838FEFDF91A9
:103E8000CF911F910895FF920F931F93CF93DF93CC
:103E9000EC01842F837009F07BC08E898B3019F47C
:103EA00081E08D871E8A8E89F98481111AC08D85E3
:103EB0008823B9F0FB01878190852F8138852817E9
:103EC00039077CF4245F3F4F2817390754F081E00D
:103ED0008E8B1D8681858F1514F083E001C08DEFD8
:103EE0008E87042F1F8148E06F2D812F98850E94B7
:103EF0002C19811115C0F2948FE0F822E12FE29580
:103F0000EF70F7E0FF9EE00D1124F0E080917B015F
:103F1000E058FE4FE80FF11D80818D7F843079F4E9
:103F20008A859B8598878F838C8589872E898D8547
:103F30009E85211123C081958D8791959E87498506
:103F40008E85480F8D856F817885680F711D87FD7F
:103F50007A9520E0CE010E943E13E9890E2E000CD6
:103F6000FF0BEE52F94FE491E88F802F90E001971C
:103F70006EE170E00E9479376F8B0AC021E08111F9
:103F800020E02D8781E0911180E08E871E8AD7CFB7
:103F90008FEFDF91CF911F910F91FF900895CF93F5
:103FA000DF93FB0126812231C1F4EC011C8A1B8ABC
:103FB0001A8A0E94FD23898582958F70EF81E29590
:103FC000EF70F7E08F9FE00D1124F0E080917B010E
:103FD000E058FE4FE80FF11D10828FEFDF91CF9177
:103FE00008956F3F11F460917B01DC01AD56BF4F26
:103FF0009C0125583E4F87E070E045E09C91973149
:1040000099F413969C91139792959F701196EC9149
:104010001197E295EF70989FE00D1124F0E0E058C1
:10402000FE4FE60FF71F40835D96A217B30731F7E7
:104030000895FC01ED56FF4F85589E4F2FEF3081BC
:10404000343109F420837D96E817F907C1F7089504
:10405000FB0126812E3F39F48285938590878783E3
:104060008485818720C02131F1F4FC012489222339
:10407000D1F0148A80919F068730A9F4E6EAF6E031
:104080008081883119F48685813069F07D9687E0DA
:10409000EE38F807A9F783E196E00E9419208CEA30
:1040A00096E00E943D248FEF0895CF92DF92EF9229
:1040B000FF920F931F93CF93DF936F3F69F0FC0143
:1040C000ED56FF4FC0E0D0E020812F3F39F0219620
:1040D0007D96C830D105C1F78FEF20C06A017C0101
:1040E0008DE18C9F80018D9F100D1124C801835795
:1040F0009F4F8E0D9F1D0E942525F601878190857B
:104100000E0D1F1DF801EC56FF4F91838083F601C1
:104110008185F801EA56FF4F80838C2FDF91CF9184
:104120001F910F91FF90EF90DF90CF900895CF9364
:10413000DF93FC01208D213009F449C0FB01268169
:10414000223018F0213109F042C0EB01FC0121E0DE
:10415000208F86EA96E00E943D248E81813071F5A1
:1041600080919F06853051F5E6EAF6E08081853141
:1041700019F48289882359F17D9627E0EE38F207F9
:10418000A9F744E156E063E083E196E00E94552000
:10419000EDE18E9FC00111248D5E994FFC01EC561C
:1041A000FF4F20E330E03183208332962CE12083DF
:1041B0003B9625E0208310929F0609C083E196E09C
:1041C0000E9419206FEF83E196E00E94F11F8FEFAC
:1041D000DF91CF910895DC01FB01878190851796CF
:1041E0002D913C9118971F964C911F97B901640F20
:1041F000711D86179707FCF44785840F911D2817BA
:104200003907CCF42185022E000C330B19964C9102
:104210001997042E000C550B50968C91BA01680F1B
:10422000711D261737073CF48089280F311D81E066
:10423000421753070CF080E00895CF93DF93EC0111
:104240008C89811116C0CB01BE010E94EB20811127
:1042500010C08F85883019F086ED96E002C088EE98
:1042600096E09B8B8A8B81E08C8B82EB96E00E94A0
:104270003D248FEFDF91CF910895CF92DF92EF929F
:10428000FF920F931F93CF93DF936C01C62F142FD0
:10429000F22ED0E0DF15A9F0612F70E0EE24E39458
:1042A00000E020E0A6018C2F90E00E946E2F84E0B9
:1042B0008C0FD23019F4185F88EF8C0FDF5FC82F96
:1042C000E9CFDF91CF911F910F91FF90EF90DF9099
:1042D000CF900895BF92CF92DF92EF92FF920F930B
:1042E0001F93CF93DF93EC0120E440E160E070E0A6
:1042F00080E090E00E94762EC090B801BC8810E06B
:10430000DD24D394FF24F394C116C9F021E01B15DA
:1043100008F420E06D2D70E0E12C00E049E15EE062
:104320008F2D90E00E94972F84E08F0D133021F4A1
:1043300084E0D80E84EF8F0D1F5FF82EE5CFFE01CD
:10434000E25AFF4FE081EF3F89F0F0E0EE0FFF1FF0
:10435000E05BF14F45915491EE24E39400E020E0BE
:104360006FE070E087E090E00E946E2FE12C00E0AB
:1043700020E049E45EE06DE070E081E090E00E94C2
:10438000972FE091C501F0E0E854FE4F238140E310
:1043900061E081E49EE00E943D21C15ADF4F288107
:1043A0004EE160E08FE29EE00E943D21E091C50178
:1043B000F0E0E854FE4F8085882359F0EE24E39422
:1043C00020E041E25EE067E170E080E090E00E9482
:1043D0006E2FDF91CF911F910F91FF90EF90DF90A3
:1043E000CF90BF9008958F929F92AF92BF92CF923D
:1043F000DF92EF920F931F93CF93DF936C0180E7CF
:1044000090E090938D0780938C0710928E07C601E1
:1044100001960E946A2110928D0710928C0744E049
:104420005EE062E088E10E94332E8091B90188232A
:1044300061F0EE24E39400E020E04AEE5DE06CE2FF
:1044400070E086E090E00E946E2F10E0460128E6C2
:10445000820E911CC12FD0E08091BA01082E000C71
:10446000990BC817D90744F5F4018081FFE01F9F1D
:104470005001112418130CC0E12C00E020E043EEA1
:104480005DE0B501665F7F4F88E190E00E94972F65
:10449000FE01EE0FFF1FED52F24F45915491B50111
:1044A000645F7F4FEE24E39400E020E08EE190E033
:1044B0000E946E2F1F5FCECF84E490E090938D0713
:1044C00080938C0710928E070091C501043008F08C
:1044D00054C0F601E359FF4F108190907C01809009
:1044E0007D0145E15EE062E080E00E94332EC0E0A5
:1044F000D0E0AA24A394B12C28E0029FC00111248B
:10450000AC0148545E4F6A018C2F612F0E946D37B9
:104510002C2F2770F50102C0EE0FFF1F2A95E2F73E
:104520009F01FE0133E0F595E7953A95E1F7EC0D33
:10453000FD1D348D2323891202C0981621F02223F9
:1045400021F022E003C021E001C020E0682F70E0EC
:104550006E5F7F4F660F771F660F771FF4E09F9F98
:10456000C0011124E12C00E04AE05EE002960E94C6
:10457000972F2196C034D10539F6DF91CF911F9145
:104580000F91EF90DF90CF90BF90AF909F908F9062
:104590000895AF92BF92CF92DF92EF92FF920F9366
:1045A0001F93CF93DF938C01D62EFC01EB59FF4F65
:1045B000908180917D01981740F43596808120E7A5
:1045C00030E07901E81AF1080AC0F801891750F4BF
:1045D000E659FF4FE080F12C80E7E81AF108C0E0CF
:1045E000D0E01CC0EA59FF4F908180917C01981760
:1045F00038F434968081C0E4D0E0C81BD1090CC0E7
:10460000891740F4F801E659FF4FC081D0E0C0544B
:10461000D10902C0C0E0D0E0E12CF12CF0928D076E
:10462000E0928C07CC2EC0938E07F801E957FF4F1C
:104630008081882359F0E114F10421F4209711F4CA
:104640009FEF0CC080917B010E94DB19F7FC09C031
:10465000D7FD67C09FEFE114F10421F420E030E0C2
:1046600007C091E09701B0E79B02200D311D112496
:1046700030938D0720938C07209729F0E0E49E9FCC
:10468000C00D112401C0C0E0C0938E078091C50108
:10469000833031F4C8010E948632D82F882329F054
:1046A000809101010E94DB19D1E05801FDE8AF0EB5
:1046B000B11CC8E0D11105C0D50116968C91883186
:1046C00049F4D501ED91FC910190F081E02D6D2D23
:1046D000C5010995C150BDE1AB0EB11CC111EACFB6
:1046E000F0928D07E0928C07C0928E070F5F1F4FEC
:1046F0006D2DC8010E94301080E790E090938D07E7
:1047000080938C0710928E07C801DF91CF911F9183
:104710000F91FF90EF90DF90CF90BF90AF900C94EF
:104720006A21E114F10409F09CCF10928D071092D8
:104730008C0791E0A3CFFF920F931F93CF93DF934A
:10474000EC01F090BA01FF2061F180E80E948C2F0B
:104750008E0108591F4F882361F0F8018081282FAE
:1047600030E02230310514F0815001C080E0F801C2
:10477000808380E10E948C2F882379F0F80180816A
:1047800090E02F2DFF0C330B215031090196281793
:1047900039070CF4C901F8018083F80180818F5F2B
:1047A000818388E00E948C2F882309F1FE01E15A61
:1047B000FF4FDE01A759BF4F8C91808377978FEF12
:1047C0008083BE9615968D919D910D90BC91A02DE4
:1047D00080839183A283B3833C96C658DF4F888140
:1047E0009981AA81BB8180839183A283B383DF9166
:1047F000CF911F910F91FF900895E0917E01F0916C
:104800007F013296E49190917C0180917D01E99F36
:10481000800D11249091C5019111865DE82FE695D8
:10482000E695E695F0E0E854FE4F877021E030E031
:10483000A90102C0440F551F8A95E2F7CA01968567
:10484000892B86870C94411AFF920F931F93CF9365
:10485000DF93EC01F62E08811981C8010E94F4361D
:10486000F81621F06F2DC8010E94FC36CE01DF91B1
:10487000CF911F910F91FF9008950F931F93CF93A6
:104880008C01C0E080914901C81728F48C2F0E9448
:104890008617CF5FF7CF10924E0110934B01009314
:1048A0004A0110934D0100934C010E94B11781E021
:1048B00080934E01CF911F910F9108959091C50162
:1048C0009430F0F4649F800D1124E82FF0E023E091
:1048D000F595E7952A95E1F728E0929FE00DF11D07
:1048E0001124E854FE4F877021E030E0A90102C096
:1048F000440F551F8A95E2F7CA01948D892B848F46
:104900000895EF92FF920F931F93CF93DF93EC01E3
:104910008C0106591F4FF8018081825080833196A7
:104920008081882351F010822091010135974081C8
:1049300031976081CE010E94B52FF80180818111ED
:104940007DC081E0FE01EA57FF4F80837E01F5E6DE
:10495000EF0EF11CF701308120917D018E010A5983
:104960001F4FCE010196321728F421E04A8560E7F7
:1049700070E014C0231728F421E04A8560E070E05D
:104980000DC0F801308120917C016885798532174E
:1049900018F421E040E402C021E040E00E943E1310
:1049A00098898CE6891B9885292F94300CF424E093
:1049B00028172CF4953014F0892F01C084E090E082
:1049C0009987888799898CE3891B9A85292F943048
:1049D0000CF424E028172CF4953014F0892F01C032
:1049E00084E08A87F701808180937D01F8016081EE
:1049F00060937C01FE01E359FF4F40810E945E24D9
:104A00008FEF8BA7FE01E85BFF4F8083BE96DE0130
:104A1000A259BF4F8D919D910D90BC91A02D808387
:104A20009183A283B3833C96C658DF4F88819981D6
:104A3000AA81BB8180839183A283B383DF91CF91CD
:104A40001F910F91FF90EF900895DC016F3F09F4E3
:104A500072C016966C93169757961C925797589655
:104A60001C92589759961C9259975A961C925A978D
:104A70001B961C921E921A971C961C921C971D96B0
:104A80001C921D971E961C921E9724E0629FC001E7
:104A900011249C012659374EF9014491FC01E55936
:104AA000F74E8491F9013296E4915696EC9356971D
:104AB000F9013396E49191E0E11101C090E05C9638
:104AC0009C935C97942F92959F709F5F1F969C93E9
:104AD0001F974F704F5F50964C935097282F30E0A0
:104AE00094E0359527959A95E1F754962C93549731
:104AF0008F7055968C935597F6E06F9FB0011124F7
:104B0000CB018E59914FFC012591349153963C93E2
:104B10002E935297FB01EC59F14F25913491139646
:104B20003C932E931297FC0134968591949115969F
:104B30009C938E93149708953F924F925F926F9239
:104B40007F928F929F92AF92BF92CF92DF92EF921D
:104B5000FF920F931F93CF93DF93CDB7DEB760978C
:104B60000FB6F894DEBF0FBECDBF2091CD0123FF5D
:104B70000AC02AE0FC01E757FF4F20832EE636E00B
:104B8000319631832083FC01E959FF4F2081222394
:104B900019F02150208343C3562E988B8F870E9493
:104BA0001919EF85F889E857FF4F83FF37C08081D7
:104BB0008F5F8083823399F5EF85F889E15AFF4F43
:104BC0008081EF85F889E859FF4F8F3F41F0AF852D
:104BD000B889A759BF4F8C938150808301C0108240
:104BE000EF85F889EA58FF4F8BE993E29183808340
:104BF000EF85F889E858FF4F11821082EF85F88918
:104C0000EE57FF4F83EF91E2918380832F853889A0
:104C10002C573F4FD9011D921C9201C310820F8562
:104C200018890F5F1F4F452DB801C8010E947413EA
:104C3000EF85F88983A18111F2C24F01F5E28F0E51
:104C4000911C6F8478882FE5620E711C7401D70166
:104C5000ED91FC910280F381E02D452DB801C70153
:104C60000995D82E682FC7010E942525BFEFDB16B6
:104C700049F0F70187819085049790878783818524
:104C800084508187FDE1EF0EF11C6E147F04F9F66C
:104C9000AF84B8882DE8A20EB11CCF84D8883BE839
:104CA000C31A3EEFD30A7501D701ED91FC91028042
:104CB000F381E02D452DB801C7010995A701682FA3
:104CC0008F8598890E945520BDE1EB0EF11CCE1412
:104CD000DF0451F77501512CEF85F889EB59FF4F2F
:104CE000FA83E9832F8538892A593F4F3C832B83E8
:104CF0008F85988984599F4F9E838D8350E4452EDC
:104D0000AF85B889AA58BF4FB887AF83EF85F889B8
:104D1000E858FF4FFA87E9872F8538892E573F4F8C
:104D20003C872B878F8598898C579F4F9E878D87CF
:104D3000D7011696DC90BFEFDB1208C05394EDE16B
:104D4000EE0EF11CF8E05F12F3CFBFC0B801C7014F
:104D50000E94EB20882309F457C02EE0D21224C011
:104D6000D7011A968C911A97E981FA8180831C9653
:104D70008C91AB81BC818C93ED81FE814082EDE012
:104D8000FDE1AF81B885ED93FC93A985BA851D92AD
:104D90001C9223EB3CE1EB85FC8531832083AD85C0
:104DA000BE851D921C9226C0B3E1DB1621F081EF77
:104DB0008D0D8230A0F4F70184898130D9F4AF855C
:104DC000B8891B968D919C911C9719969C938E93F4
:104DD00018971D968C911D971A968C930BC0A8015D
:104DE000B701C8010E94920EA801682F8F8598898B
:104DF0000E945520D701ED91FC910480F581E02DB2
:104E0000A801B801C70109956401F60186818F3FA9
:104E100031F1B601C7010E94EB20882301F1D701CF
:104E2000ED91FC910480F581E02DA801B601C70148
:104E30000995A701682F8F8598890E945520D60172
:104E4000ED91FC910480F581E02DA801B701C60128
:104E50000995A601682F8F8598890E945520BDE18C
:104E6000CB0ED11C6C147D0481F6F701868189304C
:104E700009F064CF6501312C5314F9F0D601169670
:104E80008C918930D1F4B601C7010E94EB208823B0
:104E9000A1F0D701ED91FC910480F581E02DA801EE
:104EA000B601C7010995D601ED91FC910480F58109
:104EB000E02DA801B701C60109953394BDE1CB0EE1
:104EC000D11CE8E03E12D8CF39CFEF85F889E85BF6
:104ED000FF4F8081823159F4EF84F888F2E4EF0EBD
:104EE000F11CB701C8010E94EB2081114FC18091D4
:104EF000FA05811107C0B80184EF95E00E94EB200C
:104F000081114AC1AF85B8891A96DC901A97189614
:104F1000ED90FC90199740E06D2DC7010E942C196F
:104F200030917B01882309F44FC0EF85F88995857E
:104F300023854485892F82958F70E22FE295EF704B
:104F4000F7E08F9FE00D1124F0E0E058FE4FE30FF3
:104F5000F11D8081F7FE0AC08823A9F08B30F1F0A3
:104F6000833009F459C18C3021F556C130E7E3167E
:104F7000F1044CF0882339F08B3081F03EEF380F8C
:104F80003230B8F449C1D7FE0BC08823C1F13EEFDF
:104F9000380F3230A0F18C3061F431C0D7FC09C039
:104FA0005FE35D1564F5382F3D7F49F18B5082300A
:104FB00030F1AF85B88918962C93189719964C93B1
:104FC00019971A969C931BC0D2944FE0D422EE2DD1
:104FD000E295EF70B7E0DB9EE00D1124F0E0E058C1
:104FE000FE4FE30FF11D80818D7F843041F4EF850A
:104FF000F889838594859187808785858287AF85A9
:10500000B8891A96BC901A9718968D909C9019970B
:1050100040E06B2DC4010E942C19882309F474C050
:10502000EF85F889EB59FF4F7F012F8538892A5981
:105030003F4F690197FE04C090917D01915007C0D8
:10504000B0E78B16910454F090917D019F5F90839F
:1050500090917C01D6019C9390E715C0B7FE07C0E4
:1050600090917D01908390917C01915009C0BFE3A4
:10507000BB1574F490917D01908390917C019F5FAA
:10508000D6019C9390E4EF85F889E659FF4F908311
:105090009091C501933021F48F8598890E948632C2
:1050A000EF85F889E957FF4F808340910101F601B0
:1050B0006081D7018C910E94421981E0EF85F889C7
:1050C000E559FF4F808381E894E2EF85F889EA583B
:1050D000FF4F91838083EF85F889E858FF4F118255
:1050E000108289EC92E2EF85F889EE57FF4F9183A9
:1050F0008083EF85F889EC57FF4F11821082EF858E
:10510000F889E757FF4F1082EF85F88985891816CF
:10511000FCF010820E94411A84E09CE1EF85F8893E
:10512000EA58FF4F91838083EF85F889E858FF4F55
:10513000118210828AED9CE1EF85F889EE57FF4FCE
:1051400091838083EF85F889EC57FF4F118210829D
:10515000EF84F888FCE8EF0EF11CD7018C919FEFEB
:10516000980F943008F05BC0EF85F889ED56FF4F3B
:105170002F85388925583E4F90819650983008F4F5
:105180004EC07D962E173F07B9F70DC0A801B70195
:10519000C8010E94920EABCEA80164EF75E0C80171
:1051A0000E94920EAFCE813039F48F8598890E948B
:1051B00019200E94FD232DC0823029F0843031F067
:1051C00024E0D22E05C095E0D92E02C086E0D82E6C
:1051D000A80163E08F8598890E945520EF85F889A2
:1051E0002DE1829FE00DF11D1124FA83E983EC5635
:1051F000FF4F80E390E091838083E981FA81EA5652
:10520000FF4F8CE1808389819A818F559F4FDC010C
:10521000DC92F701108203C0D7FEC2CEB8CE6096F2
:105220000FB6F894DEBF0FBECDBFDF91CF911F91B7
:105230000F91FF90EF90DF90CF90BF90AF909F9035
:105240008F907F906F905F904F903F900895CF9395
:10525000DF93EC0126E040E760E070E080E090E062
:105260000E94762EC657DF4F4881598161E081E068
:10527000DF91CF910C94332EDF92EF92FF920F9338
:105280001F93CF93DF93EC01162F8091C5018330DC
:1052900031F4CE010E948632D82E882331F08091DD
:1052A0007B010E94DB19DD24D3947E018DE8E80E9A
:1052B000F11C08E0D11005C0D70116968C918831F9
:1052C00049F4D701ED91FC910190F081E02D612F1F
:1052D000C70109950150BDE1EB0EF11C0111EACFA8
:1052E0007E01EFEFEE1AFE0A612FC7010E94301017
:1052F000EDA1FEA10190F081E02D612FCE018596F8
:105300000995CE018E5B9F4FDC01ED91FC910190E0
:10531000F081E02D612F0995612F84EF95E00E94C7
:10532000761EFE01E757FF4F8081882329F08150C8
:105330008083CE010E94272980E790E090938D071B
:1053400080938C0710928E07C701DF91CF911F9138
:105350000F91FF90EF90DF900C946A21CF93DF9331
:105360001F92CDB7DEB76983DC01ED91FC9102801D
:10537000F381E02D41E050E0BE016F5F7F4F099562
:105380000F90DF91CF91089583E08093E9008091A1
:10539000F200882319F08AE38093E8000895FC0165
:1053A0008485958597FD0BC09FB7F89482E0809324
:1053B000E9008091F2009FBF90E0019608959FB7A9
:1053C000F89482E08093E9008091F2009FBF90E022
:1053D00008954091750150917601209173013091AB
:1053E000740142175307B4F49091E8009570E1F30B
:1053F0009091E80092FD19C08093F10080917501B1
:105400009091760101968F739927892B19F48EEF6D
:105410008093E800809175019091760101969093B8
:1054200076018093750181E0089580E00895DF9210
:10543000EF92FF920F931F93CF93DF93D82E8A01A1
:105440007B01E40EF51EEB01CE15DF0571F0D7FEF2
:1054500003C0FE01849101C088810E94E929219640
:105460008111F2CF8FEF9FEF01C0C801DF91CF9183
:105470001F910F91FF90EF90DF900895615030F0F1
:105480002091F100FC0120830196F8CF289884E652
:105490008093790108950E94CA3290E008950F9395
:1054A0001F93CF93DF931F92CDB7DEB78C01FC0122
:1054B0008485958597FF0EC0CE0101960E949C328F
:1054C000019719F4898190E002C08FEF9FEFF801F6
:1054D00095878487F801848595850F90DF91CF911A
:1054E0001F910F910895CF93DF931F92CDB7DEB731
:1054F000FC018485958597FD05C02FEF3FEF35872B
:1055000024870BC0CE0101960E949C32019719F4AA
:10551000898190E002C08FEF9FEF0F90DF91CF91D4
:1055200008950F931F93CF93DF931F92CDB7DEB7EC
:1055300082E0898342E450E068EF7EE080E80E94E8
:10554000172A0E94DB32DC0112960D911C911397F1
:105550000115110589F0D801ED91FC910280F381CC
:10556000E02DBE016F5F7F4FC801099597FD04C014
:10557000F80100851185ECCF89810F90DF91CF91E3
:105580001F910F9108951F920F920FB60F92112441
:105590008F939F938091E1009091E100937F90938E
:1055A000E10083FF0FC01092E90091E09093EB00BF
:1055B0001092EC0092E39093ED0010927A0198E043
:1055C0009093F00082FF20C093E09093E9009091C7
:1055D000F200992319F09AE39093E80090917801F2
:1055E000992339F090917801915090937801992303
:1055F00089F190917901992339F090917901915035
:1056000090937901992341F184FF10C08091E200C9
:105610008E7E81608093E2008091E1008F7E809396
:10562000E100809172018E7E806111C080FF16C002
:105630008091E2008E7E80618093E2008091E100A3
:105640008E7E8093E100809172018E7E81608093D6
:10565000720104C05D9ACDCF289AD6CF9F918F91C9
:105660000F900FBE0F901F9018951F920F920FB6BC
:105670000F921124CF92DF92EF92FF920F931F931C
:105680002F933F934F935F936F937F938F939F934A
:10569000AF93BF93EF93FF93CF93DF93CDB7DEB775
:1056A0006C97DEBFCDBF1092E9008091E80083FFC8
:1056B000FBC168E0CE0145960E943E2A82EF8093AE
:1056C000E8008D8987FF05C09091E80090FFFCCF2E
:1056D00003C09EEF9093E800982F907609F0C6C023
:1056E0009E894F89588D2F89F88C91110CC0803874
:1056F00029F4809171018093F10002C01092F100B1
:105700001092F10045C1913051F4811141C14130F5
:10571000510509F03DC1809171018D7F0BC093301F
:1057200061F4811135C14130510509F031C18091D9
:1057300071018260809371012BC1953049F4809191
:10574000E80080FFFCCF822F80688093E30020C1B7
:10575000963009F05EC00B8D1C8D22E01092E9009E
:105760001092760110927501F21232C010927401FB
:10577000109273010E94912A99E0BE016F5F7F4FE2
:10578000DB01E92F1D92EA95E9F79983FA8291E00E
:105790009E8390EA98879AEF9987209175013091BE
:1057A0007601275F3F4F3C832B838D831092E90066
:1057B0001092760110927501109374010093730199
:1057C00049E050E080E00E94172A0E94912AE0C040
:1057D00010937401009373010E94DB32DC01129676
:1057E0000D911C9113970115110509F4BBC0D80147
:1057F000ED91FC910480F581E02DBE016B5E7F4F41
:10580000C8010995009709F0C7C0F8010085118506
:10581000EACF973009F445C1983021F481E08093B4
:10582000F100B6C0993009F0B3C0837009F039C1F6
:10583000E0E2F1E081E031E096E32081211109C04E
:105840008EE78093EA001092EA008F8980937A01B4
:105850009FC08093E9003093EB0021912093EC00EE
:105860009093ED008F5F873041F7EACF8B8D9C8D51
:105870001092E900109276011092750190937401D4
:1058800080937301898D811153C08E899D89913ACE
:1058900049F4813209F005C147E050E067E071E06A
:1058A00080E0BBC0913209F0FCC0833269F48F897B
:1058B000988DA0E0B0E08093030190930401A09341
:1058C0000501B093060164C0803269F48091E8005C
:1058D00082FFFCCF67E087E091E00E943E2A8BEFD9
:1058E0008093E80055C0823209F052C08F898093BE
:1058F0000E01EEEFFFE7859194918B3F9C4D19F0DF
:10590000E0E0F8E002C0EEEFFAE08091070190914C
:105910000801A0910901B0910A01803B9440A105C2
:10592000B10509F09EC080910E0180FF79C099C039
:105930000E94DB32FC01028113810115110509F47B
:10594000B0C0D801ED91FC910190F081E02DBE0135
:105950006B5E7F4FC801099581111AC0F80100855F
:105960001185EBCFF1E0FF1609F44EC0F3E0FF1212
:1059700098C08F89882309F44AC0823089F440E8AE
:1059800060E18CE59FE00E943E35882309F489C0E0
:105990008EEF8093E80088C018161906CCF381C0FA
:1059A000813029F440E86BE080E59FE0ECCF833064
:1059B00009F077C00E94DB32DC011296ED90FC907A
:1059C00013978E010F5F1F4F6801E114F10479F006
:1059D000D701ED91FC910680F781E02DB801C70158
:1059E0000995080F111DF701E084F184EECFD8016D
:1059F0001C92F60101900020E9F73197BF016C1964
:105A00007D0940E0C601BFCF6EE37FE002C06AE3DC
:105A10007FE0FB01449150E080E80E94172AB8CF54
:105A2000EE3F2AE0F20751F0808191818737A7E7A6
:105A30009A0721F09093FF0A8093FE0A87E797E781
:105A40009183808380916000809377019BE088E15F
:105A50000FB6F894A895809360000FBE90936000F5
:105A600097CF808191818737974709F091CFA8958B
:105A700080916000886180936000809177018093BD
:105A80006000EE3FBAE0FB0739F08091FE0A90918A
:105A9000FF0A918380837CCF1092FF0A1092FE0A46
:105AA00077CF81E28093EB006C960FB6F894DEBF5F
:105AB0000FBECDBFDF91CF91FF91EF91BF91AF911D
:105AC0009F918F917F916F915F914F913F912F9116
:105AD0001F910F91FF90EF90DF90CF900F900FBE2E
:105AE0000F901F9018958F929F92AF92BF92CF9276
:105AF000DF92EF92FF926B017C010E94A6164B0190
:105B00005C01C114D104E104F104F1F00E94A61675
:105B1000DC01CB0188199909AA09BB09883E934089
:105B2000A105B10570F321E0C21AD108E108F1081E
:105B300088EE880E83E0981EA11CB11CC114D1040C
:105B4000E104F10419F7DDCFFF90EF90DF90CF90E3
:105B5000BF90AF909F908F9008958F929F92AF9239
:105B6000BF92CF92DF92EF92FF920F931F93CF934A
:105B7000DF936C017B018A0180910E01882309F477
:105B80005CC080917A01882309F457C0809172012A
:105B900080FF05C08091E00082608093E000E80112
:105BA000B12C8AEFA82E93E0892E2AE3922E20971B
:105BB00011F4BB20D9F10E94CA3281110AC0AA9403
:105BC000AA20D9F161E070E080E090E00E94732D9E
:105BD000EECF282F30E0C217D3070CF48C2F9FB7DD
:105BE000F8948092E9002091E80025FF1DC0282F3D
:105BF00030E0C21BD30BF701815020F0419140935C
:105C0000F100FACFE20EF31EBB2019F09092E800EB
:105C10000AC08091E80085FD07C09092E800BB248F
:105C2000B394209709F0B12C9FBFC1CF5D9884E653
:105C3000809378011016110644F081E090E0F6019F
:105C40009383828380E090E001C0C801DF91CF910F
:105C50001F910F91FF90EF90DF90CF90BF90AF908A
:105C60009F908F9008958F92AF92CF92DF92EF9294
:105C7000FF920F931F93CF93DF93182FD62EFA0125
:105C80008491EA0121968F3F31F1E82EF12CF594B1
:105C9000E79480FF04C08CEF20E338E103C080E08C
:105CA0002CE238E160918E076D0D680F80918C07B2
:105CB00090918D07812CAA24A394C12C00E044E389
:105CC00058E1810F911D17FD9A950E943311FE0135
:105CD00084911B5FD7CFDF91CF911F910F91FF90E0
:105CE000EF90DF90CF90AF908F900895CF92DF929A
:105CF000EF92FF920F931F93CF93DF9330918E0714
:105D0000630F711D37FD7A95E0918C07F0918D0737
:105D10008E0F9F1F7C01E40EF11C8B01020F111DE1
:105D200050E124E2C22E28E1D22E8E159F053CF5CB
:105D30009B0177FF02C020E030E0F801013411053B
:105D400014F0E0E4F0E02E173F07BCF48038910532
:105D500088F4E901F6015C9FD001A0781124A80F16
:105D6000C770EC0FF11D4491AC50BE4F4095EC91C3
:105D70004E234C932F5F3F4FE0CF0196D6CFDF915C
:105D8000CF911F910F91FF90EF90DF90CF900895EA
:105D900065E070E080E090E00C94732D1F93CF934A
:105DA000DF93EC01DB01FA011F962C911F972695DA
:105DB00017968C911797280F8781281B87858695C2
:105DC000281B50968C915097869519969C91890F17
:105DD0009185891B90899695891B622F022E000C54
:105DE000770B77FF03C0719561957109482F082ED5
:105DF000000C550B57FF03C05195419551094617AB
:105E000057072CF430E0121634F020EF08C01816B3
:105E100024F030EF03C020E102C030E120E0198916
:105E200088894FE3481B842F9985432F490F942F6E
:105E300047FD90E0981724F414161CF040E001C0D0
:105E4000482F8F856FE6681B862F9F81622F690F11
:105E5000962F67FD90E0981724F416161CF060E06A
:105E600001C0682F70E020E0CE010E943E13198B24
:105E7000DF91CF911F910895FB015185DC011796A9
:105E80006D917C91189719964C91199727813085BF
:105E9000FB01E21BF30B1E161F062CF46150710967
:105EA00058961C9208C0EF2B31F06F5F7F4F21E0B6
:105EB000DC0158962C93242F042E000C330B251B49
:105EC000310957FD33951216130614F4415003C0DF
:105ED000232B09F04F5F20E00C943E138F92AF927A
:105EE000CF92EF920F93E9E8F7E03581630F0380DB
:105EF000F481E02D88248A94AE2CC02EE22E01E09D
:105F000020E030E08E0F9F1F0E9433110F91EF9021
:105F1000CF90AF908F90089520919607282329F471
:105F200090919507982381E009F480E008958F927D
:105F3000AF92CF92EF920F93E9E8F7E03581630FCC
:105F40000380F481E02D88248A94AE2CC02EE22EAA
:105F500000E020E030E08E0F9F1F0E9433110F9170
:105F6000EF90CF90AF908F9008952F923F924F92E5
:105F70005F926F927F928F929F92AF92BF92CF92D9
:105F8000DF92EF92FF920F931F93CF93DF93CDB7E2
:105F9000DEB72B970FB6F894DEBF0FBECDBF8C01D6
:105FA0002B83FC01EF59FF4F90818181E92FF82F5E
:105FB000E40FF11DE40FF11D85919491FC01E60FB2
:105FC000F11DE60FF11D85919491F801E359FF4F02
:105FD0002081A62F429FA00D11241C012FEF221A11
:105FE000320AFC0184919091C5019111BBC19A2F95
:105FF000977021E030E001C0220F9A95EAF7A6954C
:10600000A695A695B0E0A854BE4F1E96FC91F2232B
:10601000F98368012CE8C20ED11CF6011082280118
:10602000FBE84F1AFEEF5F0AF20110821A82612C20
:10603000282F30E03D832C834DE1742E9B81892FE6
:1060400090E09F838E83E251F140F987E887E62C48
:10605000062C000CFF082C813D81E216F3061CF093
:106060002DE18FEF21C1F101F491FA87FF71FB87D8
:106070002A852295269527702A877E9C50017F9C31
:10608000B00C112445013DE8830E911C800E911E39
:106090006F2FC4010E94252582E0280E311CF101DA
:1060A0003197E491A00EB11ED501AC56BF4F8E2F93
:1060B000807F90E09595879511969C938E9312968C
:1060C000EF7094E0E99FF0011124EC93F2018081DC
:1060D000811106C081E09B859B50933008F080E0E1
:1060E000F2018083FB85F43199F42A85222309F497
:1060F000D9C07E9CC0017F9C900D1124800F911F00
:10610000FC01E456FF4F38E03083319680E166C0F1
:106110009B859E3021F5E885F98540815181FA857E
:106120008F2F90E0880F991FFA01E80FF91FE49173
:106130007E9C90017F9C300D1124200F311FD901CE
:10614000A956BF4FF0E0ED93FC93FC013196E40FAC
:10615000F51F4491F901E756FF4F4083A3C02B85FB
:10616000233139F53981332309F460C07E9CC001A5
:106170007F9C900D1124800F911FFC01E156FF4F71
:1061800011821082329610823B97208122952F70C7
:106190003297E081E295EF7087E0289FE00D1124AF
:1061A000F0E0E058FE4F2E813F81E20FF31F108296
:1061B00079C03B853330A1F47E9CC0017F9C900D5B
:1061C0001124800F911FFC01EF55FF4F2A8520837A
:1061D0003981332309F466C0339681E0808362C03D
:1061E0009B85963179F4E981E1115CC07E9CF001D8
:1061F0007F9CF00D1124E00FF11FEF55FF4F2A8512
:10620000208350C03B853F3011F0353079F48981CF
:10621000882361F07E9CF0017F9CF00D1124E00F3B
:10622000F11FED56FF4F9FEF90833CC0EA85EE23B0
:10623000C9F12E2FF6012083213099F439813323BF
:1062400089F17E9CF0017F9CF00D1124E00FF11F7D
:10625000ED56FF4F8FEF8083F6011082F1E0FA8355
:1062600021C02A8522502330E8F439813323D1F02C
:10627000F601108263E0C4010E9425257E9CC001C6
:106280007F9C900D1124800F911FFC01EC55FF4F56
:1062900021E02083709720E330E031832083329621
:1062A0003CE130836394D3CE97E096155CF0362DB5
:1062B0003203F0011124E00FF11FED56FF4F8083F0
:1062C0006394F2CF8FEF8093FA058A81882319F0C7
:1062D000C8010E941920F6018081853029F0F20161
:1062E0008081811116C040C0F981FF23C1F3F601FE
:1062F0001082F801ED56FF4FC80185589E4F21E0EE
:106300003081353109F4228B7D968E179F07C1F7B6
:10631000E6CFF981FF23E1F06B81C8012B960FB620
:10632000F894DEBF0FBECDBFDF91CF911F910F91CB
:10633000FF90EF90DF90CF90BF90AF909F908F90A5
:106340007F906F905F904F903F902F900C94F11F33
:106350008EEE92E10E943D24F801E959FF4F84E658
:10636000808302C0A65D43CE2B960FB6F894DEBFA5
:106370000FBECDBFDF91CF911F910F91FF90EF9096
:10638000DF90CF90BF90AF909F908F907F906F9055
:106390005F904F903F902F900895CF92DF92EF92B1
:1063A000FF920F931F93CF93DF93EC01D62E0E94A1
:1063B000761A8091C5018150DE01AF59BF4FFE01B1
:1063C000ED59FF4F9E0123593F4F7901833090F0E3
:1063D0001092C50186E696E190937F0180937E013D
:1063E0008AE596E18D939C938AE496E1918380837C
:1063F00087E00FC083E293E190937F0180937E0159
:1064000083E193E18D939C9383E093E19183808377
:1064100088E0F70180834091C50150E0440F551F8B
:10642000FA01E550FD4E049100937D01FA01E4501C
:10643000FD4E149110937C01C0907B014C2D612F77
:10644000802F0E9442192C2D412F602FCE010E94D7
:10645000B52F898940E2481B888960E470E0681B99
:10646000710921E0CE0101960E943E1383E08A8BE0
:106470001A8EFE01E05AFF4F108282E08D8B1BA224
:1064800031978FEF80838BA7DE01A85BBF4F8C9382
:106490008091BA01181614F481E080839E012E5871
:1064A0003F4FCE018C589F4FDE01A258BF4FFE01D7
:1064B000E058FF4FDD2059F04CE955E2E9015983DE
:1064C0004883EC01198218828CE399E20BC0188290
:1064D00048E25CE1E90159834883EC0119821882A2
:1064E00082EB9BE18D939C9311821082F701408196
:1064F00060917C0180917D01DF91CF911F910F917F
:10650000FF90EF90DF90CF900C945E24FC01ED564D
:10651000FF4F85589E4F20E03081383121F4268589
:10652000222341F021E07D96E817F907A9F781E0E1
:106530008227089581E0089520917A01211103C0F6
:106540008FEF9FEF08955FB7F89422E02093E90062
:106550002091F20030E01216130614F421E030E02E
:10656000422FFC0184E6415038F02898809379014D
:106570009091F1009193F7CF2115310521F0809191
:10658000F200882319F05FBFC90108958BE680935C
:10659000E800F9CF2FB7F89483E08093E900909159
:1065A000E800892F807295FF04C09091F20080E48A
:1065B000891B2FBF089580919F0781110DC082E034
:1065C00080939B0784E080939C0710929E07109213
:1065D0009D0781E080939F078BE997E00895FC0178
:1065E00087E191E091838083138212821582148265
:1065F0008FEF868310861782118613861286148683
:106600001786108A83E0818B138A128A148A158A6E
:10661000168A178A108E118E128E138E81E0848F47
:106620000895789484B5826084BD84B5816084BD0A
:1066300085B5826085BD85B5816085BD80916E0020
:10664000816080936E001092810080918100826051
:10665000809381008091810081608093810080918E
:10666000800081608093800080919100826080939F
:1066700091008091910081608093910080919000C1
:106680008160809390008091C10084608093C100FC
:106690008091C10082608093C1008091C1008160BF
:1066A0008093C1008091C30081608093C30080917A
:1066B000C00082608093C0008091C200816080939E
:1066C000C20080917A00846080937A0080917A0081
:1066D000826080937A0080917A00816080937A0052
:1066E00080917A00806880937A0010927A011092EB
:1066F0007101109272018091D70081608093D70060
:1067000080EA8093D80089B5806189BD89B58260AF
:1067100089BD09B400FEFDCF61E070E080E090E04B
:106720000E94732D8091D8008F7C80618093D80067
:106730008091E000807F8093E0008091E1008E7E78
:106740008093E1008DE08093E200559A209A81ECDD
:1067500080937C0085B1806F85B984B1877E84B9D0
:1067600084B1876E84B95E9A5F988AB1806D8AB968
:10677000769A6E9881B3806F81BB899880B38D7053
:1067800080BB80E58CBD81E08DBD0E94C82E5F9AE4
:106790000E94C82E5E985C98E1E6F6E08EE696E0F0
:1067A00024912EBD00000DB407FEFDCF31968E174B
:1067B0009F07B1F75C9A81E880936400809165003F
:1067C00081608093650082E090E00E94F436882327
:1067D00019F00E94261902C00E9421198FE897E043
:1067E0009093500180934F0185E00E94A2188DE0A4
:1067F0000E94A218DD24D394F12CC4EFD1E000E074
:1068000010E0EE24E3948FB7F89440916901509121
:106810006A0160916B0170916C018FBF8091980744
:10682000242F281B822F90919907992329F02093D8
:106830009A07109299071BC190919707291740F466
:106840008F5F891708F013C1D3BE889513BE0FC19F
:10685000E09299074093980780919307909194074D
:1068600001969093940780939307809102018F5F24
:106870008D3319F08093020102C0E09202018F2D46
:10688000FE0181118FEF0024819381938193819385
:106890000394D1F780919507809396070E94191968
:1068A00080939507609102012091870630918806B8
:1068B000E0918506F0918606C9019595879520FFA0
:1068C0000AC0DC01AD5EB94F2D913C91E20FF31F80
:1068D0000190F081E02D8D5E994F09958091890698
:1068E00090918A06892B21F480918B0680FF28C025
:1068F0008091850690918606A0918706B0918806C2
:106900008093810690938206A0938306B0938406B9
:106910008091890690918A06A0918B06B0918C0691
:106920008093850690938606A0938706B093880689
:1069300010928A061092890610928C0610928B068D
:106940006091020110928D0710928C0710928E07B1
:106950002091930630919406E0919106F091920671
:10696000C9019595879520FF0AC0DC01AD5EB94F3E
:106970002D913C91E20FF31F0190F081E02D8D5E8F
:10698000994F099510928D0710928C0710928E07DF
:10699000809191069091920629E28C33920721F022
:1069A00022E2893C9207B1F420919306309194063B
:1069B0002115310521F0892B69F420FD0BC0809150
:1069C0009D0690919E068E56964021F483E196E0B6
:1069D0000E9427298091950690919606892B21F493
:1069E0008091970680FF36C0809191069091920623
:1069F000A0919306B091940680938D0690938E0695
:106A0000A0938F06B093900680919506909196067C
:106A1000A0919706B0919806809391069093920664
:106A2000A0939306B0939406109296061092950642
:106A3000109298061092970680919906882351F03B
:106A400080917B019091010190937B0180930101E2
:106A500010929906FE0180E098E000800EBCF110D3
:106A6000012C019780FDFDCF0192B9F70DB40115FE
:106A7000110509F4C8CE0E940000C5CEDF92EF9246
:106A8000FF920F931F93CF93DF93D82EF92EE42E0E
:106A9000062F10E0C8010196880F0E94E92983E0C3
:106AA0000E94E929CD2DDF2D0C0F1D1FC017D10726
:106AB00089F0E7FE03C0FE01849101C088810E9435
:106AC000E929F82E80E00E94E9298F212196811181
:106AD000EDCF01C081E0DF91CF911F910F91FF9029
:106AE000EF90DF900895CF93DF931092AA07109252
:106AF000A90788EE93E0A0E0B0E08093AB07909305
:106B0000AC07A093AD07B093AE078AE291E09093F3
:106B1000A8078093A7078FEF9FEF9093B407809308
:106B2000B307CFEFC093C61884EF95E00E94EF3211
:106B300086E491E0909391078093900710929507D7
:106B40001092960780E18093970710929407109215
:106B50009307109299078CE996E19093120680931F
:106B6000110680E997E090938A0780938907109235
:106B70008D0710928C0710928E071092130684E1F5
:106B800096E00E94EF328CE391E09093150680939B
:106B9000140683E196E090933406809333061092B6
:106BA000350610923606C093370688E396E00E94B9
:106BB000EF3285E596E00E94EF32C09372061092A4
:106BC00073068EEF80931A0688E0809323068093E5
:106BD00024068EEC98E1909327068093260621E008
:106BE0004CE16CE370E084E196E00E943E13109269
:106BF00078061092790610927A0610927B06C0935E
:106C00007C0610927D0610927E0610927F061092EE
:106C100082061092810610928406109283068DEBF4
:106C20009AE19093860680938506109288061092CA
:106C3000870610928A061092890610928C0610928E
:106C40008B0610928E0610928D061092900610926E
:106C50008F0682EA9BE190939206809391061092B0
:106C60009406109293061092960610929506109232
:106C70009806109297061092990681E080939A06E2
:106C800010929B0610929F06C0E0D0E0CE01805685
:106C9000994F0E94EF326D96C83ED105B9F7DF914A
:106CA000CF9108958F929F92AF92BF92CF92DF9231
:106CB000EF92FF92CF93DF93EC01688179818A8113
:106CC0009B81611571058105910521F464E279EDDF
:106CD0008BE597E02DE133EF41E050E00E940A3769
:106CE00049015A019B01AC01A7EAB1E40E9429378E
:106CF0006B017C01ACEEB4EFA50194010E94373723
:106D0000DC01CB018C0D9D1DAE1DBF1DB7FF03C067
:106D10000197A109B04888839983AA83BB83BC01EA
:106D2000CD019F77DF91CF91FF90EF90DF90CF90D3
:106D3000BF90AF909F908F9008958F929F92AF9247
:106D4000BF92CF92DF92EF92FF9260910F0170910C
:106D50001001809111019091120161157105810559
:106D6000910521F464E279ED8BE597E02DE133EFB5
:106D700041E050E00E940A3749015A019B01AC01F1
:106D8000A7EAB1E40E9429376B017C01ACEEB4EFB5
:106D9000A50194010E943737DC01CB018C0D9D1DAC
:106DA000AE1DBF1DB7FF03C00197A109B048809376
:106DB0000F0190931001A0931101B0931201BC0137
:106DC000CD019F77FF90EF90DF90CF90BF90AF9075
:106DD0009F908F90089560930F017093100180939E
:106DE0001101909312010895F999FECF92BD81BDD2
:106DF000F89A992780B50895262FF999FECF1FBAE2
:106E000092BD81BD20BD0FB6F894FA9AF99A0FBED3
:106E100001960895052E97FB1EF400940E942137D9
:106E200057FD07D00E943C3707FC03D04EF40C946A
:106E3000213750954095309521953F4F4F4F5F4FEB
:106E4000089590958095709561957F4F8F4F9F4FD6
:106E500008950E945E37A59F900DB49F900DA49F4A
:106E6000800D911D11240895B7FF0C9429370E94BD
:106E70002937821B930B0895A1E21A2EAA1BBB1B74
:106E8000FD010DC0AA1FBB1FEE1FFF1FA217B307F6
:106E9000E407F50720F0A21BB30BE40BF50B661F0C
:106EA000771F881F991F1A9469F7609570958095D0
:106EB00090959B01AC01BD01CF010895A29FB00147
:106EC000B39FC001A39F700D811D1124911DB29F1E
:106ED000700D811D1124911D0895991B79E004C046
:106EE000991F961708F0961B881F7A95C9F7809509
:106EF000089597FB072E16F4009407D077FD09D06C
:106F00000E948D3707FC05D03EF4909581959F4FE8
:106F10000895709561957F4F0895AA1BBB1B51E1A1
:106F200007C0AA1FBB1FA617B70710F0A61BB70BF9
:106F3000881F991F5A95A9F780959095BC01CD019E
:106F40000895EE0FFF1F0590F491E02D099481E064
:0C6F500090E0F8940C94AC37F894FFCF5C
:106F5C00041C01FFFFFFFF00E10000000000000126
:106F6C0000000000000000761ED21AD41D030100A0
:106F7C00C1808100000000000000AE29AD2D4B2A1D
:106F8C00C429CF29732A4F2A000000003010741333
:086F9C00920E000000009F1698
:00000001FF
